:020000040800F2
:10000000900C0024AD020008054000088F3900085C
:10001000B9020008D9080008C94D00080000000016
:10002000000000000000000000000000B3430008D2
:10003000FF0900080000000007400008B145000863
:10004000C7020008C7020008C7020008C70200086C
:10005000C7020008C7020008C7020008C70200085C
:10006000C7020008C7020008C7020008C70200084C
:10007000C7020008C7020008C7020008C70200083C
:10008000C7020008C7020008C7020008C70200082C
:10009000C7020008C7020008C7020008C70200081C
:1000A000C7020008C7020008C7020008C70200080C
:1000B000C7020008C7020008C7020008C7020008FC
:1000C000C7020008C7020008C7020008C7020008EC
:1000D000C7020008854D0008C7020008C7020008D3
:1000E000C7020008C702000800000000C70200089D
:1000F000C7020008C7020008C7020008C7020008BC
:10010000C7020008C7020008C7020008C7020008AB
:10011000C7020008C7020008C7020008C70200089B
:10012000C7020008C7020008C7020008C70200088B
:10013000C7020008C7020008C7020008C70200087B
:1001400000000000000000000000000000000000AF
:10015000C7020008C7020008C7020008C70200085B
:10016000C7020008C7020008C7020008C70200084B
:10017000C7020008C7020008C7020008C70200083B
:10018000C7020008C7020008C7020008C70200082B
:10019000C7020008C7020008C7020008C70200081B
:1001A000C7020008C7020008C7020008C70200080B
:1001B000C7020008C7020008C7020008C7020008FB
:1001C000C7020008C7020008C7020008C7020008EB
:1001D000C7020008C7020008C7020008C7020008DB
:1001E000C7020008C7020008C7020008C7020008CB
:1001F000C7020008C7020008C7020008C7020008BB
:10020000C7020008C7020008C7020008C7020008AA
:10021000C7020008C7020008C7020008C70200089A
:10022000C7020008C7020008C7020008000000005B
:10023000C7020008C702000800000000C70200084B
:10024000C7020008C7020008C7020008C70200086A
:10025000C7020008C7020008C7020008C70200085A
:10026000C7020008C7020008C7020008C70200084A
:10027000C7020008C7020008C7020008000000000B
:10028000C702000800000000C702000800000000CC
:1002900000000000C7020008DFF80CD000F036FABA
:1002A0000048004755570008900C00240648804736
:1002B00006480047FEE7FEE7FEE7FEE7FEE7FEE74B
:1002C000FEE7FEE7FEE7FEE7B545000899020008F5
:1002D0002DE9F05F0546002092469B46884606467B
:1002E000814640241BE0284641464746224600F00E
:1002F00045F853465A46C01A914110D31146184644
:10030000224600F02CF82D1A67EB01084F462246D2
:100310000120002100F023F817EB00094E41201EB8
:10032000A4F10104DFDC484631462A464346BDE8D5
:10033000F09F30B50B46014600202022012409E041
:1003400021FA02F59D4205D303FA02F5491B04FA8E
:1003500002F52844151EA2F10102F1DC30BD202A6D
:1003600004DB203A00FA02F1002070479140C2F10C
:10037000200320FA03F3194390407047202A04DB3E
:10038000203A21FA02F00021704721FA02F3D0400E
:10039000C2F1200291400843194670472DE9FE4FF3
:1003A000804681EA0300C00F0C46009021F0004116
:1003B00023F00045B8EB0200A94105D24046214692
:1003C00090461C460B46024623F00040104347D09F
:1003D000270DC7F30A00C3F30A510290401A019097
:1003E00040286BDAC3F3130040F4801B0098924658
:1003F00020B10023D2EB030A63EB0B0B01985946A3
:10040000C0F140025046FFF7AAFF06460D4650468F
:100410005946019A00F08CF910EB08006141002464
:1004200087EA115284EAE7731A4340D0009A62B314
:10043000019A012A4FEA075215DC001B61EB020109
:100440004FF0004202EA0752CDE90042001C41F59C
:10045000801132462B4600F08CF903B0BDE8F08FD6
:1004600040462146F9E7001B61EB0201001C41F503
:10047000801300185B412018A2F5001747EB030119
:1004800040EAD570B6196D4111E06D084FEA3606A5
:1004900045EAC0754FEA0752001B61EB0201001CE0
:1004A00041F5801149084FEA3000001951413246A8
:1004B0002B4603B0BDE8F04F00F04CB90098012284
:1004C00040000023D0EB020263EBE073009821466A
:1004D0004FEAE074B8EB000061EB0401E9E783F058
:1004E00000435BE781F0004158E72DE9FE4F81EAC8
:1004F000030404F0004421F0004100944FF0000B8D
:1005000023F0004350EA01045ED052EA03045BD0BA
:10051000C3F30A54C1F30A552C44A4F2F3340194F2
:10052000A0FB0254C1F3130141F48011C3F3130380
:1005300043F4801301FB024400FB034E840A970A34
:1005400044EA815447EA8357A4FB076802958D0A61
:1005500005FB07854FEA932C04FB0C542705029DED
:100560004FEA065847EA1637B5EB08056EEB070C5D
:10057000870E920E47EA811742EA8312A7FB020117
:10058000B6EB0B0164EB00042B0D43EA0C335E1851
:1005900044EB1C50DA465146E7FB0201C5F3130455
:1005A0004FEA0B3343EA14534FEA0432019C43EA07
:1005B0000603A4F10C040294009CCDE900B400F001
:1005C000D8F803B0BDE8F08F00200146F9E72DE927
:1005D000F04D81EA030404F0004B21F0004514467D
:1005E0004FF0000A23F0004150EA050220D054EAFF
:1005F00001021DD0C5F30A570246C5F31303C1F328
:100600001300C1F30A5640F4801543F48013A7EB9E
:100610000608101BD64608F2FD3873EB050002D31E
:1006200008F1010801E092185B41B8F1000F03DA0C
:1006300000200146BDE8F08D00204FF480110646F1
:1006400084460EE0171B73EB050705D3121B63EB03
:10065000050306434CEA010C49084FEA30009218A2
:100660005B4150EA0107EDD152EA030012D082EA61
:10067000040083EA0501084305D0101BAB4106D2F4
:100680000122002306E000224FF0004302E06FF059
:10069000010253101AEB06004CEB085110EB0A0054
:1006A00041EB0B01BDE8F04D00F054B8C1F30A5224
:1006B000C1F3130140F2FF3341F480119A4202DA90
:1006C00000200146704740F233439A42A2F233427F
:1006D00002DC5242FFF752BEFFF741BE30B5041EA6
:1006E00071F1000404DB4FF00044404264EB01016F
:1006F000141E73F1000405DB1C464FF00043524208
:1007000063EB0403994208BF904230BD064C074D8D
:1007100006E0E06840F0010394E8070098471034D1
:10072000AC42F6D3FFF7BCFD987B0008B87B00080D
:10073000202A06DBCB17203A41FA02F043EAE073A5
:1007400006E041FA02F3D040C2F120029140084392
:100750001946704710B5141E73F1000408DA401CE6
:1007600041F1000192185B411A4301D120F00100D0
:1007700010BD2DE9F04D92469B4611B1B1FA81F2C0
:1007800002E0B0FA80F220329046FFF7E8FD04461E
:100790000F4640EA0A0041EA0B0153465A46084315
:1007A00013D0114653EA010019D0C8F14002504657
:1007B000FFF7E4FD05460E46504659464246FFF710
:1007C000CEFD084305D0012004E020463946BDE8AF
:1007D000F08D0020054346EAE0762C4337430A9823
:1007E0006305E40AA0EB08000022FD0A44EA47542E
:1007F0000A3002D500200146E9E7010510196941D8
:10080000DDE9084500196941BDE8F04DA2E770B582
:1008100004460068816801F00301012925D10168BF
:10082000C90722D0816801F00D0101290FD181682B
:1008300041F00201816021680320086001F01EFA86
:1008400005460EE001F01AFA401B022809D9606D36
:1008500040F010006065A06D40F00100A06501202F
:1008600070BD20688068C007ECD1002070BD00001A
:1008700070B504460068816801F00301012902D1C6
:100880000168C90723D18168124A114210D18168D9
:1008900041F00101816001F0F1F9054612E0816843
:1008A00041F00101816001F0E9F9401B022809D9FA
:1008B000606D40F010006065A06D40F00100A06523
:1008C000012070BD20680168C943C907E7D1002035
:1008D00070BD00003F000080FEE70000F0B5BFF3F0
:1008E0004F8FBFF36F8F1D4900200860BFF34F8FFC
:1008F000BFF36F8F1A4C216841F400312160BFF3C0
:100900004F8FBFF36F8F164970310860BFF34F8F61
:10091000081F006843F6FF75104E1036C0F34E31C5
:10092000C0F3C90305EA4112184642EA80773760EE
:10093000401EFAD2491EF5D2BFF34F8F206840F413
:1009400080302060BFF34F8FBFF36F8F03484C3070
:10095000016841F004010160F0BD000050EF00E0CB
:1009600014ED00E02DE9F0430D4F00241D4616461E
:100970008846814604EB041017F81010B14209D1E3
:1009800007EB40014878A84204D1891C42464846FA
:1009900000F02AF8641CA4B2382CEBD3BDE8F08335
:1009A000DC7000082DE9F0430E4F00241D4616466A
:1009B0008846814604EB840000EB441017F81010C1
:1009C000B14209D107EB40014878A84204D1891C03
:1009D0004246484600F008F8641CA4B2092CE9D34A
:1009E000BDE8F083B2780008002310B504E011F8E8
:1009F000014B5B1C00F8014B9342F8D310BD7047CC
:100A0000F0B51C46094B0A4F164685B04FF0000C56
:100A100010251A885B883F88121A5B1A8DE8F0103F
:100A200092B29BB200F0BAF905B0F0BD7C0200248E
:100A3000260000242DE9FF411C46084B16460027DE
:100A400010251A885B88121A5B1A8DE8F00092B2A2
:100A50009BB203F0FBFCBDE8FF8100007C02002498
:100A60002DE9FF411C46084B1646002718251A8819
:100A70005B88121A5B1A8DE8F00092B29BB203F009
:100A8000E5FCBDE8FF8100007C0200242DE9F04177
:100A90001546DFF85C8001220C46064640461703E7
:100AA000394601F0E5F8052000F0D6F9032003F0FF
:100AB000C9FBC4F3074003F0C5FBC4F3072003F0F0
:100AC000C1FBE0B203F0BEFB002405E0FF2003F011
:100AD000B9FB3055641CA4B2AC42F7D300223946AE
:100AE000404601F0C5F8BDE8F041052000F0B4B97A
:100AF0000004025830B40C460178202A1AD009DCD0
:100B00000C2A0DD0102A13D0182A17D10C4801FB3B
:100B1000030108E0302A0FD0402A0FD10948F6E738
:100B2000594301F50021204630BC1A46FFF7AEBFFD
:100B30000548ECE70548EAE70548E8E730BC7047B8
:100B400000120800009208000008080000260800B3
:100B50000048080030B40C460146007815464A7833
:100B6000812809D3402A07D3FF2A05D0FF2803D0C4
:100B70007F2A0CD2403A0BE00022104603E0521CC0
:100B800092B204F8010B9A42F9D330BC7047413A53
:100B90008138C0B2D1B2C0EB401202EB801001EB41
:100BA000400159430C2D0CD0102D0CD0182D0DD018
:100BB000202DEAD101F56011204630BC1A46FFF71E
:100BC00065BF044800E004480144F5E701F5ED1174
:100BD000F2E700000014090000DD1100AFF300800F
:100BE00070B586B04FF6FF7002F002FF00206C4631
:100BF00005462554401CC0B21828FAD311222046BD
:100C00000021FFF743FF10216B464FF4784608465A
:100C10003246FFF7F5FE00202554401CC0B21828CC
:100C2000FAD3082268461421FFF730FF20216B46D3
:100C300010203246FFF7E4FE00202554401CC0B2CD
:100C40001828FAD3082268461E21FFF71FFF30211B
:100C50006B4610203246FFF7D3FE4FF4FA6004F0E3
:100C600051FD06B070BD2DE9F04FC1B01C461646CF
:100C70000D4682468946580701D0012100E0002137
:100C800001EBD40061080C2C10FB01F0834609D065
:100C9000102C07D0182C05D0202C03D0302C01D0DC
:100CA000402C2DD10346224669463046FFF722FFED
:100CB000002022E01DF808700026380601D54A9A67
:100CC00002E04C9820B94B9A2946504602F0F2FEB9
:100CD00078066D1CADB2070EA5EB0900A04205D148
:100CE0000AF101004D461FFA80FA03E0761CB6B205
:100CF000082EE2D308F1010080B258458046D9D3CE
:100D000041B0BDE8F08F2DE9F04FA1B01F46154668
:100D10000C4682468946580701D0012100E0002197
:100D200001EBD7000C2F10FB07F0834605D0102FE6
:100D300003D0182F01D0202F2DD103463A46694603
:100D40002846FFF707FF002022E01DF80860002575
:100D5000300601D52A9A02E02C9820B92B9A214618
:100D6000504602F0A7FE7006641CA4B2060EA4EB67
:100D70000900B84205D10AF101004C461FFA80FA79
:100D800003E06D1CEDB2082DE2D308F10100C0B202
:100D900058458046D9D321B0BDE8F08F2DE9FF4FEB
:100DA00083B09B460E46044680468A46DDE91075B0
:100DB0000020814620E0B9F1000F23D005994FF0C3
:100DC000000908EB0100401BA04202DA70194446FA
:100DD00086B20AEB0B00401BB04210DB12AB93E86B
:100DE00007002B468DE807003A4631462046FFF7BC
:100DF0008AFF601984B2BF1C38780028DBD107B0A5
:100E0000BDE8F08F802801D90120D2E7059A08EBD0
:100E10000201A1EB5501A14202DA711944468EB2DA
:100E20000AEB0B01491BB142E9DB0D280FD012ABD5
:100E300093E807002B468DE807003A4631462046E6
:100E4000FFF711FF04EB550084B27F1CD4E7701943
:100E5000444686B27F1CF5E7002206E00021491CCB
:100E6000C9B26429FBD3521CD2B28242F6D3704776
:100E700000B587B0694600900120019005200290DE
:100E80000020039004900590074800F09DF8064864
:100E900000F02CFD04480A2100F08CFC024800F010
:100EA00027FB07B080B200BD900100242DE9F0417E
:100EB00000250E4607462C4608E03846FFF7D8FFC7
:100EC0000544052004F01EFC641CE4B2B442F4D3D3
:100ED000B5FBF6F080B2BDE8F08170B4164602783A
:100EE0001D464378812A0C4610D3402B0ED3FF2B8E
:100EF0000CD0FF2A0AD00C2D11D0102D11D0182D96
:100F00000DD13146204670BCFFF74CBD002108468C
:100F100003E0491C04F8010BC9B2B142F9D370BC1B
:100F200070473146204670BCFFF71CBD2DE9F041EB
:100F3000044690F850000025164601280F460CD0B4
:100F4000012084F850002046FFF761FC0100606D2D
:100F50002A4605D040F0100031E00220BDE8F081C3
:100F600020F4885040F0020060652068836823F018
:100F70008043334383602068836823F480333B439A
:100F800083602068836843F00043836020684FF4E7
:100F90007A460CE06D1CB54209D3606D20F002006A
:100FA00040F010006065012084F85020D6E7836887
:100FB000002BEFDB606D20F0020040F00100606567
:100FC000084684F85020C9E72DE9F84F0023FC4C6F
:100FD0004FF0804E9B46009390F85020012A28D075
:100FE000012580F850500268966876077ED4D6694D
:100FF000AA460F78BD402E43D6614A681F254FF49C
:10100000F868052A18D20668376B98FAA8FCBCFA6B
:101010008CFC02FB0CFC05FA0CF598FAA8FCAF431B
:101020000D68BCFA8CFC02FB0CF295402F43376331
:1010300049E00220BDE8F88F0A2A16D20668776BCD
:1010400098FAA8FC521FBCFA8CFC02FB0CFC05FAB7
:101050000CF598FAA8FCAF430D68BCFA8CFC02FBB7
:101060000CF295402F4377632DE006680F2A15D2C6
:10107000B76B98FAA8FC0A3ABCFA8CFC02FB0CFC91
:1010800005FA0CF598FAA8FCAF430D68BCFA8CFC85
:1010900002FB0CF295402F43B76314E0F76B98FA0C
:1010A000A8FC0F3ABCFA8CFC02FB0CFC05FA0CF510
:1010B00098FAA8FCAF430D68BCFA8CFC02FB0CF25A
:1010C00095402F43F763026895684FF038064FF05C
:1010D000070915F00C0F7DD10D680A2D1BD39769F8
:1010E00096FAA6FC0A3DBCFA8CFC00E0C9E105FBBF
:1010F0000CF809FA08FC96FAA6F827EA0C07D1F8CA
:1011000008C0B8FA88F805FB08F50CFA05FC47EAB0
:101110000C07976117E0576996FAA6FCBCFA8CFC9D
:1011200005FB0CF809FA08FC96FAA6F827EA0C0762
:10113000D1F808C0B8FA88F805FB08F50CFA05FCE8
:1011400047EA0C07576102684D69D7684FF0F84CC1
:10115000C7F382077F00BD400F69012F4AD0022FDD
:101160006AD0032F7DD0042F7CD0156E9CFAACF88A
:1011700005F0F8470D68B8FA88F805FA08F5AF42A7
:1011800003D1156E25F0004515660268556E9CFA70
:10119000ACF805F0F8470D68B8FA88F805FA08F5D4
:1011A000AF4203D1556E25F0004555660268956E35
:1011B0009CFAACF80F68B8FA88F805F0F84507FA19
:1011C00008F7BD4203D1956E25F00045956602688B
:1011D000D56E00E02FE09CFAACFC05F0F8470D68F6
:1011E000BCFA8CFC05FA0CF5AF4224D1D56E25F083
:1011F000004589E0176E9CFAACFC07F000480F68C8
:10120000BCFA8CFC07FA0CF72F4348EA0708C2F82F
:101210006080026815690F7E25F400653D43156105
:101220004A7E002A0268156E02D045F0004501E0B2
:1012300025F00045156668E0576E9CFAACFC07F097
:1012400000480F68BCFA8CFC07FA0CF72F4348EAF9
:101250000708C2F86480026815690F7E25F480557E
:1012600001E00FE031E045EA470515614A7E002ABA
:101270000268556E02D045F0004501E025F00045BA
:10128000556642E0976E9CFAACFC07F000480F6888
:10129000BCFA8CFC07FA0CF72F4348EA0708C2F89F
:1012A0006880026815690F7E25F4005545EA8705B8
:1012B00015614A7E002A0268956E02D045F000450D
:1012C00001E025F0004595661FE0D76E9CFAACFC66
:1012D00007F000480F68BCFA8CFC07FA0CF72F43A4
:1012E00048EA0708C2F86C80026815690F7E25F489
:1012F000804545EAC70515614A7E002A02683FF429
:1013000075AFD56E45F00045D5660268956805F065
:101310000305012D02D11568ED0761D1CD68754532
:1013200007D052F8C06F0F780AFA07F5AE4316607F
:101330003CE052F8C07F91F800C00AFA0CF52F4348
:1013400017600A680568092A18D3AF6996FAA6FCDF
:10135000093ABCFA8CFC96FAA6F602FB0CF8B6FA2F
:1013600086F609FA08FC724327EA0C07D1F808C090
:101370000CFA02FC47EA0C07AF6117E06F6996FAB6
:10138000A6FC521CBCFA8CFC96FAA6F602FB0CF8E2
:10139000B6FA86F609FA08FC724327EA0C07D1F878
:1013A00008C00CFA02FC47EA0C076F61054E05689D
:1013B000054FB54201D0BD420AD1044A09E0000000
:1013C0000060025800200240002102400023024039
:1013D000444A0968122904D0112907D013290AD0D8
:1013E00054E0D2F808C04FEA0C2C08E0D2F808C04C
:1013F0004FEACC1C03E0D2F808C04FEA4C2CBCF1F9
:10140000000F43DBD5F808C00CF0030CBCF1010F52
:1014100004D1D5F800C05FEACC7C32D1B54210D1FE
:10142000D6F8087107F00307012F03D1D6F8006141
:10143000F60726D1A66806F00306012E2AD12668F3
:101440001DE0BD42B76807F003070BD1012F02D1A1
:101450003768FF0715D1A76807F00307012F06D1EA
:10146000276802E0012F02D13768FF0709D1D6F8BB
:10147000087107F00307012F0CD1D6F80061F607B9
:1014800008D0416D41F020014165012380F850B042
:101490001846CFE512290AD011291CD01329F5D1FD
:1014A000A542F3D1916841F480019160EEE7A54235
:1014B000ECD1916841F4000191600B490B4A096835
:1014C000B1FBF2F1C1EB0111C90000E0491E00912E
:1014D0000029FBD1DAE7A542D8D1916841F08071AB
:1014E000E3E70000006302580800002480841E0027
:1014F0000068006C70470000F8B54FF0000504006C
:101500002E46009502D0606D10B107E00120F8BDB5
:10151000204600F021F9A66584F8506020688168B3
:10152000890003D5816821F00051816020688168BD
:10153000C90010D4816841F0805181607D487E49A6
:101540000068B0FBF1F000EB8000400000E0401EBE
:1015500000900028FBD120688168C90008D4616D23
:1015600041F010016165A16D41F00101A165012506
:10157000616DC9067ED481684907FBD4616D41F075
:10158000020161656D4A6E4E904201D0B04201D1B8
:101590006C4900E06C49836803F00303012B02D11E
:1015A0000368DB0739D1694B904210D1D2F80801AA
:1015B00000F00300012803D1D2F80001C0072CD1AC
:1015C000986800F00300012821D118681DE0B0429E
:1015D000906800F003000BD1012802D11068C00709
:1015E0001BD1986800F00300012806D1186802E0BA
:1015F000012802D11068C0070FD1D2F8080100F00D
:101600000300012803D1D2F80001C00705D1886882
:10161000626820F47C1010438860A1684FF4803326
:10162000206B627D93FAA3F308434FF40051B3FAA1
:1016300083F391FAA1F1B1FA81F18A40217F01FA95
:1016400003F31A431043012909D14FF46022216AA0
:1016500092FAA2F2491EB2FA82F291400843616AFC
:10166000012903D0A26A0AB1114308432168CA685C
:10167000374B00E056E01A400243CA602068816898
:1016800011F00C0F28D14FF48042217D92FAA2F282
:10169000B2FA82F29140E26A1143C26844F2030353
:1016A0009A430A43C26094F8390001281CD020688C
:1016B000016921F00101016120680169626B21F07B
:1016C00070411143016194F8380001282068816855
:1016D0001AD021F480718160E06801282068016BD4
:1016E00021F00F0113D015E0D4E91010A28F0123CF
:1016F0000143A06C03EB02421043014320680269DE
:10170000144B1A401143D6E741F48071E3E7A26914
:10171000521E11430163606D20F0020040F0010091
:10172000606504E0606D40F01000606501252846AA
:10173000F8BD00000800002480841E000020024044
:10174000002102400023024000630258006002585A
:1017500003C0F0FF1EF800FC144800B587B0016814
:1017600041F020010160006800F0200005900F4862
:101770000830016841F004010160006800F00400D5
:1017800005900A488038016821F4403141F4003165
:101790000160012000900320019000200290044885
:1017A000694600F06DF907B000BD0000D84402584A
:1017B000000802582DE9F04704460069DFF81C9143
:1017C000012608280F4622D020684946884202D0C8
:1017D000434A90421DD1D1F80823D20619D0D1F83E
:1017E000082302F01F02052A13D0D1F8081301F0D4
:1017F0001F0109290DD03B488168C1F381310229BD
:101800000AD08068C0F38130032805D00BE008259A
:101810000AE0C068C00706D0606D40F02000606537
:101820000120BDE8F087042500F028FA804611E089
:10183000781C0FD02FB100F021FAA0EB0800B842BD
:1018400008D9606D40F004006065002084F8500005
:101850000320E6E7206800682842E9D02068016894
:10186000090700D400264946884224D01E4A9042E7
:1018700021D0D1F80823D2061DD0D1F8082302F0D8
:101880001F02052A17D0D1F8082302F01F02092AE7
:1018900011D0C968082D10D04A0401D40422026076
:1018A000606D40F400706065B6B12068C06810F4E7
:1018B000406F04D010E0C168ECE70822EFE788042D
:1018C0000AD4606D20F480706065606DC00403D43C
:1018D000606D40F0010060650020A2E7002002403A
:1018E00000210240002302400060025870B5044607
:1018F00000688068400767D494F8500001280AD037
:10190000012084F850002046FEF7B2FF01004FF09E
:10191000000202D045E0022070BD606DC00404D515
:10192000A06D20F00600A06500E0A265606D40F6A5
:101930000163984340F480706065254B20689842AD
:1019400006D0244DA84203D0D3F80853ED0603D1A6
:10195000656D25F4801565651C2505602068984235
:1019600022D01D4DA8421FD0D3F80853ED061BD03E
:10197000D3F8085305F01F05052D15D0D3F80853EB
:1019800005F01F05092D0FD0606D40F480106065D3
:10199000D868800105D5606D20F4005040F4805077
:1019A000606584F8502010E0C3689B0105D5636D25
:1019B00023F4005343F48053636584F85020826815
:1019C00042F00402826000E00221084670BD00007F
:1019D00000200240002102400060025810B528B1EA
:1019E00090F83510022903D080214165012010BDF7
:1019F0001D4A4FF4956301688C189C4207D8042255
:101A000080F83520086820F00100086029E00C68A3
:101A100024F00E040C6001680A440A6822F00102F6
:101A20000A60016E0A6822F480720A6090F85C30E5
:101A3000012202FA03F10D4B1960D0E919134B6032
:101A4000C16E31B10B6823F480730B60D0E91C13B5
:101A50004B60002180F8341080F83520016D01B111
:101A60008847002010BD0000F0FFFDBF045402585D
:101A70000248016841F001010160704720040058EC
:101A80002DE9F84F6C4C00224FF0B04A4FF0010B9B
:101A90004FF0030E4FF00F090B680BFA02F73B40B3
:101AA000BB4270D14D68022D01D0122D12D1D50844
:101AB00000EB850CDCF820605507ED0E09FA05F8FF
:101AC00026EA0806D1F8108008FA05F848EA060860
:101AD000CCF82080D0F80080560091F804C00EFAAF
:101AE00006F50CF0030C28EA05080CFA06FC4CEA93
:101AF000080CC0F800C0D1F804C0BCF1010F08D038
:101B0000BCF1020F05D0BCF1110F02D0BCF1120FD5
:101B100016D1D0F808C0D1F80C802CEA050C08FAD0
:101B200006F848EA0C08C0F80880D0F804C02CEA8F
:101B3000070C0F79C7F30017974047EA0C07476077
:101B4000C768AF438D68B5403D43C5604D68ED0043
:101B50006BD53A4D2E6846F002062E602D6822F0B5
:101B6000030606F1B04605F002050095D6F808C454
:101B700095072F0F09FA07F52CEA050C304DA842FE
:101B800002D100252EE050E02E4DA84201D10125C2
:101B900028E02D4DA84201D1022523E02B4DA8427B
:101BA00001D103251EE02A4DA84201D1042519E0E8
:101BB000284DA84201D1052514E0274DA84201D1A6
:101BC00006250FE0254DA84201D107250AE0244D46
:101BD000A84201D1082505E0224DA84201D10925DE
:101BE00000E00A25BD4045EA0C05C6F80854256802
:101BF0004E689D43F60300D51D43256065684E6819
:101C00009D43B60300D51D436560DAF80050564683
:101C10004F689D43FF0200D51D43356075684F68CE
:101C20009D43BF0200D51D437560521C102AFFF46E
:101C300033AFBDE8F88F000080000058F44402582C
:101C4000000002580004025800080258000C025814
:101C5000001002580014025800180258001C0258C4
:101C6000002002580024025842694A4042617047ED
:101C70000AB10183704741837047000001488068C2
:101C8000704700001800002402488168027811445F
:101C90008160704718000024032010B500F058F848
:101CA0000F2000F007F808B1012010BD00F022F865
:101CB000002010BD70B50D4D04464FF47A712878A0
:101CC000B1FBF0F00A490968B1FBF0F001F08CFCBF
:101CD00048B9102C07D200222146501E00F018F8F7
:101CE00000206C6070BD012070BD00001800002451
:101CF000080000247047002809DB012100F01F02C2
:101D000091404009800000F1E020C0F800117047C8
:101D10000E4BF0B41B68C3F30223C3F10704042C79
:101D200000D904241D1D072D01D2002300E0DB1E75
:101D3000012606FA04F56D1E0D409D409E40761E5C
:101D4000164045EA0601F0BC03F054B80CED00E083
:101D5000064A00F0070110684FF6FF03184040EAFA
:101D60000120034908431060704700000CED00E0BB
:101D70000000FA0510B500F0B3FE084909684FF4F9
:101D8000807292FAA2F201F47061B2FA82F2D1404A
:101D9000034A515CC8400349086010BD184402580A
:101DA000F45800080800002410B500F053FE07495D
:101DB0000968102292FAA2F201F07001B2FA82F2DE
:101DC000D140034A515CC84010BD00002044025875
:101DD000F4580008364930B50A68096812F0030261
:101DE000344BC1F305311B68334C03F010032468F6
:101DF000DFED320AB7EE001AC4F3CC0414FB03F390
:101E000000EE103A2E4BB8EE400A07D02D4C012AB6
:101E100001D0022A4AD0B4FBF1F10BE0244C283C5B
:101E200022689506284A03D52468C4F3C104E24019
:101E3000B2FBF1F101EE901A1968B8EE612AC1F314
:101E4000080101EE901A1968F8EE611A40EE201AA6
:101E500031EE810A22EE000AC1F34621491C00EE50
:101E6000901AF8EE600A80EE201AFCEEC10AC0ED6E
:101E7000000A1968C1F30641491C00EE901AF8EEF9
:101E8000600A80EE201AFCEEC10AC0ED010A196852
:101E9000C1F30661491C00EE901AF8EE600A80EE6C
:101EA000201ABCEEC10A80ED020A30BD074ABFE726
:101EB000284402582C4402583C440258000000397F
:101EC0003844025800093D000090D00340787D015D
:101ED000364930B50A68096812F00302344BC1F381
:101EE00005511B68334C03F480732468DFED320A1C
:101EF000B7EE001AC4F3CC0414FB03F300EE103A5F
:101F00002E4BB8EE400A07D02D4C012A01D0022AF0
:101F10004AD0B4FBF1F10BE0244C283C2268950632
:101F2000284A03D52468C4F3C104E240B2FBF1F1AE
:101F300001EE901A1968B8EE612AC1F3080101EEAA
:101F4000901A1968F8EE611A40EE201A31EE810AF3
:101F500022EE000AC1F34621491C00EE901AF8EE69
:101F6000600A80EE201AFCEEC10AC0ED000A196872
:101F7000C1F30641491C00EE901AF8EE600A80EEAB
:101F8000201AFCEEC10AC0ED010A1968C1F306610E
:101F9000491C00EE901AF8EE600A80EE201ABCEEA2
:101FA000C10A80ED020A30BD074ABFE72844025843
:101FB0002C4402584444025800000039404402585E
:101FC00000093D000090D00340787D012DE9F84FD5
:101FD0000446006800252E46010104F12400FE4F4E
:101FE000DFF8F88300901DD5606E50B1B0F5801F0A
:101FF0000CD0B0F5001F0ED0B0F5401F1DD001254C
:102000000FE0386840F40030386016E00221201DEF
:1020100001F0FAFF03E00098022102F06DF80500DC
:102020000BD02E462088C00523D5606D05281ED212
:10203000DFE800F00C11161B1B00D8F80010626ED0
:1020400021F440111143C8F80010EBE7386840F460
:102050000030386009E00021201D01F0D5FF03E0C9
:102060000098002102F048F805466DB100E0012516
:102070002E432088800528D5A06D80281ED00CDC3A
:1020800090B140280ED114E0D8F80010626D21F014
:1020900007011143C8F80010EBE7C02813D0B0F5D2
:1020A000807F10D001250FE0386840F400303860A0
:1020B00009E00021201D01F0A7FF03E000980021A6
:1020C00002F01AF8054685B12E432088DFF81093F8
:1020D00040052CD5D4F8A400B0F5800F20D00DDC3D
:1020E000A0B1B0F5001F0FD115E0D8F80010A26D17
:1020F00021F4E0711143C8F80010E6E7B0F5C00F15
:1021000013D0B0F5000F10D001250FE0386840F46F
:102110000030386009E00021201D01F075FF03E068
:102120000098002101F0E8FF054675B12E43208894
:1021300000052DD5D4F8A800B0F1007F21D00EDC29
:10214000A8B1B0F1807F10D116E0D9F80010D4F812
:10215000A42021F460011143C9F80010E7E7B0F1B1
:10216000407F13D0B0F1806F10D001250FE03868A8
:1021700040F40030386009E00021201D01F044FFE8
:1021800003E00098002101F0B7FF05466DB12E4332
:10219000206880011FD5A06CD8B110280FD020284E
:1021A00012D0302815D0012514E0D9F80010D4F849
:1021B000A82021F0E0611143C9F80010E8E7386871
:1021C00040F40030386004E00221201D01F01CFFC3
:1021D00005466DB12E432088C0042BD5E06DB0F5C7
:1021E000005F20D00DDCA0B1B0F5805F0FD115E00D
:1021F0007A48001F0168A26C21F030011143016090
:10220000E9E7B0F5405F13D0B0F5804F10D001255D
:102210000FE0386840F40030386009E00021201DEC
:1022200001F0F2FE03E00098002101F065FF054691
:1022300085B12E432088800429D5206EB0F5403F1B
:1022400023D010DC08B3B0F5803F14D0B0F5003FC8
:102250000FD115E0D8F80010E26D21F4E0411143F0
:10226000C8F80010E6E7B0F5802F0ED0B0F5A02F2B
:102270000BD001250AE00121201D01F0C5FE03E07D
:102280000098012101F038FF05468DB12E432088CA
:1022900040042AD5D4F8AC00B0F1405F23D010DC64
:1022A00008B3B0F1805F14D0B0F1005F0FD115E03A
:1022B000D8F80010226E21F4E0211143C8F8001074
:1022C000E5E7B0F1804F0ED0B0F1A04F0BD0012563
:1022D0000AE00121201D01F097FE03E00098012192
:1022E00001F00AFF05466DB12E43208800041FD57A
:1022F000E06ED8B1B0F1805F0ED0B0F1005F10D0C9
:10230000012514E0D9F80010D4F8AC2021F0E04108
:102310001143C9F80010E8E7386840F4003038602D
:1023200004E00121201D01F06FFE05466DB12E4332
:102330002068C0011ED5606CD0B101280ED00228E3
:1023400011D0032814D0012513E0D8F80010E26E54
:1023500021F040511143C8F80010E9E7386840F413
:102360000030386004E00221201D01F04DFE0546DA
:1023700075B12E432068DFF86CB040025AD51A4878
:10238000016841F480710160FFF778FC82460EE03D
:102390001248001F0168626C21F0030111430160C3
:1023A000E8E7FFF76BFCA0EB0A0064283AD80E4878
:1023B0000068C005F5D5B5BB094818300068B4F809
:1023C000B01000F4407001F44071884219D0044804
:1023D000183001680AE000002C44025850440258AA
:1023E000584402581044025800480258026821F428
:1023F000407142F480320260026822F4803202604E
:102400000160D4F8B000B0F5807F22D1FFF736FC30
:10241000824609E0FFF732FCA0EB0A0141F2883066
:10242000814201D9032504E0FE4800688007F1D508
:102430007DB12E432078DFF8F0A3C0073CD0A06F19
:10244000182837D025DC78B3082828D0102824D1C4
:102450002BE0D4F8B000C0F3012103290ED0DBF843
:10246000001021F47C51CBF80010EE480168B4F85C
:10247000B020C2F30B0211430160DBE7DBF8002060
:10248000EA4B22F47C5203EA10100243CBF80020FE
:10249000EBE720280ED028280CD001250BE00121E5
:1024A000201D01F0B1FD04E004E00098012101F0DD
:1024B00023FE05465DB12E43207880071ED5606F50
:1024C000062819D2DFE800F0160C11161616DAF8F5
:1024D0000010A26F21F038011143CAF80010EBE799
:1024E0000121201D01F090FD03E00098012101F081
:1024F00003FE054675B100E001252E432078400714
:102500001FD5D4F89000062819D2DFE800F0160C89
:1025100011161616DAF80010626F21F00701114348
:10252000CAF80010EAE70121201D01F06DFD03E06B
:102530000098012101F0E0FD05469DB100E0012574
:102540002E43207880062BD5D4F88C00B0F1405F64
:1025500024D011DC10B3B0F1805F15D0B0F1005F72
:1025600010D116E0D9F80010D4F8902021F007011E
:102570001143C9F80010E4E7B0F1804F0ED0B0F17C
:10258000A04F0BD001250AE00021201D01F03CFDE9
:1025900003E00098022101F0AFFD05468DB12E4306
:1025A000207840062BD5D4F89800B0F5406F24D0A1
:1025B00011DC10B3B0F5806F15D0B0F5006F10D1FD
:1025C00016E0DAF80010D4F88C2021F0E041114335
:1025D000CAF80010E4E7B0F5805F0ED0B0F5A05F58
:1025E0000BD001250AE00021201D01F00DFD03E0C4
:1025F0000098022101F080FD05468DB12E43207820
:1026000000062BD5D4F89C00B0F5C04F24D011DCC7
:1026100010B3B0F5005F15D0B0F5804F10D116E0C3
:10262000D9F80010D4F8982021F4E0511143C9F8EA
:102630000010E4E7B0F5004F0ED0B0F5204F0BD0FE
:1026400001250AE00021201D01F0DEFC03E00098D6
:10265000022101F051FD054665B32E4320780007A5
:102660000BD5D4F88000B0F5805F2DD0DAF80020CB
:1026700022F440520243CAF800202078C0060BD54D
:10268000D4F89400B0F5807F24D0D9F8002022F44B
:1026900040720243C9F80020206800032CD5D4F80A
:1026A000A000E8B1B0F5803F1FD0B0F5003F21D0C9
:1026B000012520E0D9F80010D4F89C2021F46041D5
:1026C0001143C9F80010C9E70098022101F014FD78
:1026D0000643D2E70098022101F00EFD0643DBE736
:1026E0000021201D01F090FC03E00098022101F080
:1026F00003FD054685B12E432068400322D5D4F85A
:102700008400B0F5801F11D0B0F5001F13D0B0F5D4
:10271000401F15D0012514E0D9F80010D4F8A020EE
:1027200021F440311143C9F80010E5E7386840F45E
:102730000030386004E00098012101F0DDFC05461E
:1027400055B12E432068C0031CD5E06C70B1B0F5C4
:10275000803F10D0012514E0DAF80010D4F884206E
:1027600021F440111143CAF80010EBE7386840F437
:102770000030386004E00221201D01F045FC0546D0
:10278000C5B12E432068800004D50098022101F0D5
:10279000B3FC0643206880031BD5E06FB8B1B0F5E9
:1027A000807F10D0B0F5007F11D0B0F5407F0ED003
:1027B00001250DE01C4808380168E26C21F48031E5
:1027C00011430160DEE7386840F40030386045B3FB
:1027D0002E432068C00207D5D8F80000226F20F0F1
:1027E00000401043C8F800002068C00008D5DBF89E
:1027F0000010D4F8B42021F480411143CBF800102C
:102800002068800207D5D8F80010A26E21F08071F0
:102810001143C8F800102068400014D5DBF8001000
:1028200006E01EE07044025854440258CFFFFF00F7
:1028300021F40041CBF80010DBF80010D4F8B820E8
:102840001143CBF800102068002806DA0A48016816
:10285000226D21F04051114301605EB10120BDE8BD
:10286000F88FDAF80010E26F21F440711143CAF8D2
:102870000010AEE70020F2E74C4402582DE9F04783
:10288000DFF8BC9104460E46D9F8000000F00700BE
:10289000B0420CD2D9F8001021F007013143C9F839
:1028A0000010D9F8000000F00700B0427ED1207877
:1028B000DFF89081800707D5D8F80010E26821F092
:1028C0000F011143C8F800102078C00762D0D8F873
:1028D0000010A26821F470611143C8F80010594932
:1028E0006068183902281CD003281DD00968012807
:1028F0001DD04907002960DA524F083F396821F09E
:10290000070101433960FFF7B9F90546606841F2F4
:102910008831022813D003281ED001288A4627D0E8
:1029200034E009688903E5E709688901E2E7C90538
:10293000E0E7FFF7A3F9411B514501D923E08A469F
:102940003868C0F3C2000228F3D123E0FFF796F9FC
:10295000411B514501D916E08A463868C0F3C200D0
:102960000328F3D116E0FFF789F9411B51450AD836
:102970003868C0F3C2000128F5D10BE0FFF77EF9FB
:10298000411B514502D90320BDE8F087386810F09B
:10299000380FF3D1D9F80010484601F00701B142D1
:1029A0000DD9016821F00701314300E005E0016025
:1029B000006800F00700B04201D00120E4E7207871
:1029C000400707D5D8F80010226921F070011143A3
:1029D000C8F80010207801071B4805D50168626916
:1029E00021F07001114301602178C90605D5016805
:1029F000A26921F4E061114301602078800607D5C7
:102A00001149091D0868E26920F070001043086050
:102A100000F066F8D8F800104FF4807292FAA2F233
:102A200001F47061B2FA82F2D140084A515CC840A8
:102A3000074908600F20FFF73DF90020A4E70000D8
:102A400000200052184402581C440258F458000850
:102A50000800002410B5FFF78DF908490968012224
:102A600092FAA2F201F00F01B2FA82F2D140044AC6
:102A7000515CC8400349086010BD0000184402586A
:102A8000F45800080C00002410B5FFF7E3FF0749D5
:102A90000968102292FAA2F201F07001B2FA82F2F1
:102AA000D140034A515CC84010BD00001C4402588C
:102AB000F458000810B5FFF7CDFF074909684FF437
:102AC000807292FAA2F201F4E061B2FA82F2D1408D
:102AD000024A515CC84010BD1C440258F45800081A
:102AE0003548F0B50068364D10F03801334809D04C
:102AF0000411082904D0334E10290BD018290BD00B
:102B00002046F0BD29688906FBD52968C1F3C101BB
:102B1000C840F0BD3046F0BD274918310A68096841
:102B200012F00302284BC1F305111B68274F03F075
:102B300001033F68DFED260AB7EE001AC7F3CC07A2
:102B400017FB03F300EE103A224BB8EE400A06D012
:102B5000012A01D0022A2BD0B4FBF1F008E02A6848
:102B6000920603D52A68C2F3C102D040B0FBF1F04F
:102B700001EE900A1868B8EE612AC0F3080001EE71
:102B8000900A1868F8EE611A40EE201A31EE810AB8
:102B900022EE000AC0F34620401C00EE900AF8EE38
:102BA000600A80EE201ABCEEC10A10EE100AF0BDD9
:102BB000B6FBF1F0DCE70000104402580090D003AF
:102BC0000044025840787D012C4402583444025895
:102BD00000000039304402582DE9F05F04460078C7
:102BE000DFF8FC8341F28839DFF8F8A3FE4DC00717
:102BF0004ED0D8F800104046C1F3C20102291AD0C5
:102C00000068C0F3C200032805D1DAF8000000F024
:102C1000030002280FD06068B0F5803F12D010B1D9
:102C2000B0F5A02F19D0286820F4803028602868DB
:102C300020F4802009E02868800329D560680028F6
:102C400074D025E0286840F480302860606890B136
:102C5000FFF714F806464F4609E0286840F4802044
:102C60002860EFE7FFF70AF8801BB8427DD8286894
:102C70008003F7D50CE0FFF701F806464F4604E065
:102C8000FEF7FCFF801BB842F0D828688003F7D419
:102C90002078D64F80075AD5D8F8001040464FF418
:102CA0007C3B11F0380F13D00068C0F3C20003283A
:102CB00003D1DAF8000080070AD0E068A8B32968D9
:102CC00021F0190101432960FEF7D8FF06461DE0F7
:102CD0002868400702D5E0680028B1D02868E1687C
:102CE00020F0190008432860FEF7C8FF064604E0FC
:102CF000FEF7C4FF801B0228B8D828684007F7D524
:102D000007E0FEF7BBFF801B0228AFD8286840070A
:102D1000F7D538689BFAABF220F47C312069B2FA1F
:102D200082F290400143396011E000E0AEE0286893
:102D300020F001002860FEF7A1FF064604E0FEF740
:102D40009DFF801B022891D828684007F7D420787F
:102D5000C00655D5D8F8001040464FF0F84BC1F3E7
:102D6000C201012917D0006800E0EDE0C0F3C20005
:102D7000032805D1DAF8000000F0030001280AD08A
:102D8000E069002828682CD040F080002860FEF719
:102D900075FF064616E02868C00502D5E069802860
:102DA00074D138689BFAABF220F0F841206AB2FA8D
:102DB00082F290400143396022E0FEF75FFF801B02
:102DC000022899D82868C005F7D538689BFAABF275
:102DD000216AB2FA82F220F0F8409140084338604C
:102DE0000EE020F080002860FEF748FF064604E071
:102DF000FEF744FF801B022887D82868C005F7D457
:102E00002078000724D5774F60694C370028386850
:102E10000FD040F001003860FEF730FF064604E0B6
:102E2000FEF72CFF801B02288DD838688007F7D565
:102E30000EE020F001003860FEF720FF064604E0B7
:102E4000FEF71CFF801B02287ED838688007F7D465
:102E50002078800623D5A069002828680FD040F488
:102E600080502860FEF70AFF064604E0FEF706FFE2
:102E7000801B022868D828688004F7D50FE020F46A
:102E800080502860FEF7FAFE064605E0D6E0FEF721
:102E9000F5FE801B022857D828688004F7D42078D4
:102EA000400744D5524F386840F480703860FEF7D0
:102EB000E5FE064604E0FEF7E1FE801B642843D8E9
:102EC0003868C005F7D5474FA068483701280AD0B1
:102ED00008B1052811D0386820F001003860386842
:102EE00020F0040002E0386840F001003860A0687B
:102EF00088B1FEF7C3FE064609E0386840F00400DA
:102F00003860F0E7FEF7BAFE811B49451CD83868E7
:102F10008007F7D50BE0FEF7B1FE064604E0FEF7AA
:102F2000ADFE811B49450FD838688007F7D4606A29
:102F3000F0B3D8F80010C1F3C20103297ED00228F3
:102F4000286820F0807000E079E0286003D0FEF768
:102F500095FE044687E0FEF791FE064604E0FEF784
:102F60008DFE801B02287BD828688001F7D4DAF810
:102F7000001040F2F3329143E26A41EA0211A26A80
:102F80001143CAF8001094F834004FF4FE02218E69
:102F90004002491EA0F5007080B2C1F30801084349
:102FA000218F491E02EA0141084394F83C1000E0D9
:102FB0005CE0491E120202EA016108430949083136
:102FC00008600B1D19684FF6F872A06C914392FAD5
:102FD000A2F2B2FA82F2904001431960014809E07E
:102FE000104402582844025800440258044402582D
:102FF00000480258001D0168226C21F00C011143A9
:1030000001600168626C21F00201114301600168F6
:1030100041F480310160016841F4003101600168D0
:1030200041F480210160016841F0010101602868DC
:1030300040F080702860FEF721FE01E018E00FE00C
:10304000044604E0FEF71AFE001B022808D8286890
:103050008001F7D50AE0FEF711FE001B022802D915
:103060000320BDE8F09F28688001F4D40020F8E731
:103070000120F6E72DE9F05F04004FF000053DD098
:10308000DFF8C4812068714E714F4045A36A06D0B5
:10309000B04204D0B84202D0E1680F292ED8E26BCA
:1030A0004FF0010B0BEB521CE26802F10801C9085A
:1030B000404501FB0CF105D0B04203D0B84201D02D
:1030C00008291BD8404503D0B04201D0B84201D1F5
:1030D000102913D84FF480094B4512D1404507D031
:1030E000B04205D0B84203D0206BB0F5702F05D8A0
:1030F000256B05B91504B2EB154F02D90120BDE8C7
:10310000F09F94F881004FF0000A20B9204684F81F
:1031100080A000F09FF8022084F8810020680168F8
:1031200021F001010160A069B0F1806F09D16068F0
:10313000484506D1A06B20B92068016841F4805150
:103140000160A16AE0690843E16B29430843E16833
:10315000084321688860616A606BA2690843A16BBB
:10316000114308432169084361690843216A084300
:1031700061680843E16C0843A1680843A16C0843F7
:10318000A16D08432168C860A06A484529D1206C18
:1031900001282068016827D021F400410160606C9B
:1031A00001282068016822D021F480410160206854
:1031B000404506D0B04204D0B84202D0B5F5702FD9
:1031C00018D0404503D0B04201D0B84202D1B5F585
:1031D000F81F0FD0016821F4005101602168E06AF6
:1031E0000864606850B119E041F40041D6E741F449
:1031F0008041DBE7016841F40051EEE7A06A30B995
:103200002068816821F4C05141F400618160206828
:10321000816821F4C06141F4806181602068016DA2
:1032200021F0010101656068400206D52068C1688F
:10323000626D21F000411143C160C4F884A084F89C
:1032400081B000205BE70000003001400038004002
:10325000003C0040164800B5B5B0016841F00201DD
:103260000160006800F002003490114808300168E5
:1032700041F480410160006800F4804034904FF4D4
:1032800080500090002017906846FEF79FFE4FF494
:1032900060402F9002203090012031900320329026
:1032A0000520339003482FA9FEF7EAFB35B000BD97
:1032B000E0440258000402582DE9F84F044690F803
:1032C00080001F4692460A9D01288B4613D04FF07E
:1032D000010984F88090FEF7D1FC94F8812006461D
:1032E0000020012A4FF480010ED062688A4209D181
:1032F000A2683AB902E00220BDE8F88F94F8812074
:10330000042A01D0022136E0BBF1000F32D0BAF11D
:10331000000F2FD077B394F88120042A02D0052221
:1033200084F881208046C4F88400C4F864A0A4F81E
:103330006A70A4F86870C4F85CB0A4F86270A4F86D
:10334000607020676067206842686FF30F023A433D
:1033500042602068026842F00102026060688842B0
:1033600004D12068016841F400710160E0680F2811
:1033700040D848E0012184F880000846BCE7B4F852
:10338000620070B12068416989070AD5E16D09685A
:103390000162E06D001DE065B4F86200401EA4F813
:1033A0006200B4F86A0080B12068416948F20802FE
:1033B00011420AD0006B616E0860606E001D60668D
:1033C000B4F86A00401EA4F86A00681C12D0FEF728
:1033D00055FC801BA8420DD3204600F05BFF84F80B
:1033E0008080D4F8840040F48070C4F8840084F8AD
:1033F0008190EBE0B4F862000028C0D1B4F86A0014
:103400000028BCD1C8E0072849D8BDE0B4F8620064
:10341000F0B12068416989071AD5B4F86210012912
:103420000BD9E16B49B1E16D09680162E06D001DE6
:10343000E065B4F86200801E08E0E16D098801844F
:10344000E06D801CE065B4F86200401EA4F86200E4
:10345000B4F86A00E0B12068416911F4604F17D0F8
:103460004169090409D5006B616E0860606E001D3A
:103470006066B4F86A00801E08E0008E616E088005
:10348000606E801C6066B4F86A00401EA4F86A0092
:10349000681C04D0FEF7F2FB801BA8429CD2B4F853
:1034A00062000028B2D1B4F86A000028AED173E0FF
:1034B000B4F8620080B32068416989072CD5B4F85C
:1034C000621003290CD9E16B402909D9E16D096823
:1034D0000162E06D001DE065B4F86200001F19E0B4
:1034E000B4F8621001290BD9E16B49B1E16D09888B
:1034F0000184E06D801CE065B4F86200801E09E084
:10350000E16D097880F82010E06D401CE065B4F8AA
:103510006200401EA4F86200B4F86A0068B3206834
:10352000416911F4604F28D04169090409D5006B45
:10353000616E0860606E001D6066B4F86A00001F6E
:1035400019E0416901F4C041B1F5005F09D9008E6D
:10355000616E0880606E801C6066B4F86A00801E30
:1035600009E090F83000616E0870606E401C606683
:10357000B4F86A00401EA4F86A00681C04D0FEF784
:103580007DFB801BA84289D2B4F8620000288FD14D
:10359000B4F86A0000288BD1002233460821204667
:1035A000009500F0E6FE28B1D4F8840040F0200039
:1035B000C4F88400204600F06DFE84F8808084F812
:1035C0008190D4F8840000283FF4D8AE012093E61F
:1035D0004FF0E0210428086903D020F004000861BE
:1035E000704740F00400FAE7401EB0F1807F10B54C
:1035F00001D3012010BD4FF0E02460610F2160175E
:1036000001F0F8FB0020A06107202061002010BD20
:103610007047704790F8791090F87A000843704727
:1036200070B502680446D0691368916810F00F0FF6
:1036300064D0594D03F490760D40354376D0C507DC
:1036400007D0DD0505D501251562E26F42F00102C4
:10365000E267820708D5CA0706D0256802222A62D7
:10366000E26F42F00402E267420708D5CA0706D0BB
:10367000256804222A62E26F42F00202E267020732
:103680000ED503F0200201F080552A4352EAC172A0
:1036900006D0256808222A62E26F42F00802E2673B
:1036A000E26F002A3AD0800608D503F0200001F02E
:1036B0008051084302D0204601F068F8E06F00070F
:1036C00003D42068806840062AD5204601F050F8CF
:1036D0002068816849061ED5816821F0400181601B
:1036E000606FC0B12D490165606FFEF777F9002862
:1036F00014D0606F016DBDE870400847850615D590
:1037000003F0200501F0805635430FD02046BDE878
:10371000704001F03BB82046FFF77BFF70BD05E02D
:103720002046FFF776FF0020E067F7E7C6024FF07C
:1037300020050CD54E020AD5E803106284F87950B2
:1037400084F87A502046BDE87040FFF761BF060656
:103750000AD503F0800601F400010E4304D0204690
:10376000BDE8704001F0A2BA41060BD5590609D553
:103770001168204621F04001116084F8795000F072
:1037800005F9CBE70002C9D55800C7D5106820F06D
:1037900080401060C2E70000010000105D47000893
:1037A00010B5040003D094F8790010B107E00120AF
:1037B00010BD002084F87800204600F027F824206F
:1037C00084F879002068016821F001010160204639
:1037D00001F018F80128EBD0606B10B1204600F022
:1037E0002BFF2068416821F4904141602068816886
:1037F00021F02A0181602068016841F00101016027
:103800002046BDE8104000F07BBF000010B5006806
:1038100086B01B49884230D11A48016841F0010145
:103820000160006800F00100059016481030016842
:1038300041F01001016000680121134C00F01000FC
:1038400005904FF4007000900220CDE90101039033
:103850000720694604902046FEF712F94FF4806174
:10386000204600916946FEF70BF92520FEF743FA42
:10387000032225201146FEF74BFA06B010BD0000CA
:1038800000100140E04402580000025890F87A30DD
:10389000202B4CD1B9B1B2B190F87830012B46D081
:1038A000012380F878304166A0F86820A0F86A20EB
:1038B000FF228168B1F5805F07D07F2351B1B1F15C
:1038C000805F0CD010E001207047016921B940F2FF
:1038D000FF1107E0016909BBA0F86C2004E0016951
:1038E000E1B13F21A0F86C100021C167222280F8CD
:1038F0007A2080F8781001688A6842F001028A60B4
:1039000001680A6892000CD50A6842F480720A6065
:103910000068816841F08051816006E0A0F86C3059
:10392000E2E7086840F490700860002070470220C9
:103930007047000030B50068114988420CD1114A27
:103940005088010408D411464FF00003440409785C
:1039500006D50A2901D0538030BD40F400400DE067
:103960000D2909D0084DC0F30D04401C80B2C728B2
:1039700029555080EFD830BD40F48040508030BD94
:103980000010014014000024480000247047FEE7A6
:10399000144870B586B0016841F004010160016807
:1039A00001F004010591016841F010010160006817
:1039B00000260325694600F0100005900820012428
:1039C000CDE900060848CDE90245FEF759F8202068
:1039D0006946CDE900060548CDE90245FEF750F8F5
:1039E00006B070BDE04402580010025800080258AA
:1039F0002DE9F0410D4F00240646214620467B88E4
:103A00003A8800F0BDF93D88002178884543084692
:103A100000F0A2F900F09CFA03E0304600F042FA10
:103A2000641CAC42F9D3BDE8F08100007C020024A4
:103A30002DE9F0411E490027F0222C242A252B26AF
:103A40004FF4A07338B1012817D002284FF0010CB1
:103A50001BD0032822D08F710A804B800C81002458
:103A60004D818E814B880A880021084600F088F934
:103A70002046BDE8F04100F05DB98F710B804A80AF
:103A80000C8101244D818E81ECE781F806C00A800B
:103A90004B800C8102244D818E81E3E781F806C0C2
:103AA0000B804A800C8103244D818E81DAE700006F
:103AB0007C0200242DE9F0410B4C16460F460546CA
:103AC000608900F029FA284600F0ECF9A08900F09E
:103AD00023FA384600F0E6F9208900F01DFA304656
:103AE000BDE8F04100F0DEB97C0200241A4810B5B0
:103AF00086B0016841F00201016000686946174C18
:103B000000F00200059041F20300009001200190B6
:103B10000290032003902046FDF7B2FF01222046C9
:103B20001146FEF7A5F8012220460221FEF7A0F873
:103B3000012220461103FEF79BF800F055FBA0047C
:103B400000F090FB00F00CF8012220461146FEF731
:103B50008FF806B010BD0000E0440258000402587F
:103B600070B50A4D4FF48044002221462846FEF7E6
:103B70007FF8322001F0C6FD012221462846FEF7DB
:103B800077F8BDE870401E2001F0BCBD000402586B
:103B900010B5FFF7ABFF00F07BF9322001F0B2FD6A
:103BA000362000F0B9F9002000F09AF93A2000F030
:103BB000B3F9052000F094F9B22000F0ADF90C2023
:103BC00000F08EF90C2000F08BF9002000F088F94D
:103BD000332000F085F9332000F082F9B72000F09F
:103BE0009BF9352000F07CF9BB2000F095F91920F5
:103BF00000F076F9C02000F08FF92C2000F070F969
:103C0000C22000F089F9012000F06AF9C32000F019
:103C100083F9122000F064F9C42000F07DF920201F
:103C200000F05EF9C62000F077F90F2000F058F997
:103C3000D02000F071F9A42000F052F9A12000F08A
:103C40004FF9E02000F068F9D02000F049F9042095
:103C500000F046F90D2000F043F9112000F040F982
:103C6000132000F03DF92B2000F03AF93F2000F03E
:103C700037F9542000F034F94C2000F031F91820C5
:103C800000F02EF90D2000F02BF90B2000F028F9A0
:103C90001F2000F025F9232000F022F9E12000F098
:103CA0003BF9D02000F01CF9042000F019F90C2099
:103CB00000F016F9112000F013F9132000F010F9AC
:103CC0002C2000F00DF93F2000F00AF9442000F00C
:103CD00007F9512000F004F92F2000F001F91F200E
:103CE00000F0FEF81F2000F0FBF8202000F0F8F8AC
:103CF000232000F0F5F8212000F00EF9112000F04B
:103D00000BF9782001F0FEFC292000F005F9C8200D
:103D100001F0F8FC0020FFF78BFE01220448114659
:103D2000FDF7A6FFBDE810404FF6FF70FFF760BE3D
:103D300000040258002158B1012804D0022804D000
:103D4000032805D103E0602102E0C02100E0A021AA
:103D5000362000F003B9000070B5084C0D46064649
:103D6000608900F0D9F8304600F09CF8A08900F096
:103D7000D3F82846BDE8704000F094B87C020024D7
:103D80002DE9F04104460E4F10448846401E86B28D
:103D9000C818401E85B2788900F0BEF8204600F0B1
:103DA00081F8304600F07EF8B88900F0B5F840465A
:103DB00000F078F82846BDE8F04100F073B8000044
:103DC0007C0200242DE9F84F1F460C4682468B46A4
:103DD000580700D00120790800EBD700203A10FBEB
:103DE00001F0002602F0FF09C0B2009040E00C2F65
:103DF0000FD0102F11D0182F3DD1204909EBC90049
:103E000001EB80004FF00008855D280609D50A9A6D
:103E10000BE01B4909EB4900F2E71A4901EB0910D5
:103E2000F0E70B9828B91848428821465046FFF71A
:103E300041FE6806641C050E1448A4B24088A042E6
:103E400019D9A4EB0B00B84209D10AF101005C4674
:103E50001FFA80FA0D48018851450CD906E008F197
:103E6000010000F0FF08B8F1080FCED3761CF6B2BF
:103E700000988642BBD3BDE8F88F0000806300083D
:103E80001C590008905D0008240000247C020024D6
:103E9000012010B500F040F8BDE81040322001F0DC
:103EA00031BC000070B50D4E4FF480550022044621
:103EB00029463046FDF7DCFE012230460221FDF79F
:103EC000D7FE200A00F0BEF9E0B200F0BBF92946A7
:103ED0003046BDE870400122FDF7CABE000402581A
:103EE00070B50C4D4FF480540022064621462846FA
:103EF000FDF7BEFE012228460221FDF7B9FE30463D
:103F000000F0A0F921462846BDE870400122FDF7E7
:103F1000AFBE00000004025870B50C4E4FF480553F
:103F20000022044629463046FDF7A2FE0022304614
:103F30000221FDF79DFEE0B200F084F929463046EB
:103F4000BDE870400122FDF793BE00000004025856
:103F500001480089FFF7E0BF7C02002410B50C4641
:103F6000FFF7DAFFE0B2BDE81040FFF7B9BF00008D
:103F70000E4810B586B0016841F00101016000688B
:103F800069460B4C00F001000590022000900120D2
:103F900001900290032003902046FDF771FD01225D
:103FA00020460221FDF764FE06B010BDE044025831
:103FB0000000025812480422104910B501604FF465
:103FC0004031416000218160C0E903120175012286
:103FD000417582610177C0E90812816280F838205A
:103FE0001203026380F83910C162FDF785FA0022DE
:103FF0000348BDE810401146FCF798BF002002407E
:1040000090010024704770472DE9F047DFF8E48005
:1040100004460F464FF00009D8F80000C04380075F
:1040200009D0344D283D286820F080602860FDF7D5
:1040300025FE064607E00120BDE8F087FDF71EFEDD
:10404000801B02284ED828680001F7D4D8F8001049
:10405000226821F47C3141EA0231C8F80010207A4C
:104060004FF4FE02A1884002491EA0F5007080B204
:10407000C1F308010843A189491E02EA014108432E
:10408000217C1202491E02EA0161084319491031DC
:1040900008601848001D0168626921F0C0011143E1
:1040A00001600168A26921F02001114301606FB134
:1040B0000168012F0ED041F400110160286840F022
:1040C00080602860FDF7DAFD04460DE0016841F4E8
:1040D0000021F2E741F48011EFE7FDF7CFFD001B6F
:1040E000022801D90320A7E728680001F5D5484632
:1040F000A2E70000284402582DE9F047DFF8E480E9
:1041000004460F464FF00009D8F80000C04380076E
:1041100009D0344D283D286820F080502860FDF7F4
:10412000ADFD064607E00120BDE8F087FDF7A6FDDE
:10413000801B02284ED828688000F7D4D8F80010D9
:10414000228821F07C7141EA0251C8F80010207ADF
:104150004FF4FE02A1884002491EA0F5007080B213
:10416000C1F308010843A189491E02EA014108433D
:10417000217C1202491E02EA0161084319491831E3
:1041800008601848001D0168626921F4406111430C
:1041900001600168A26921F40071114301606FB1EF
:1041A0000168012F0ED041F080710160286840F055
:1041B00080502860FDF762FD04460DE0016841F47F
:1041C0008001F2E741F40001EFE7FDF757FD001B26
:1041D000022801D90320A7E728688000F5D54846C2
:1041E000A2E700002844025810B5154C07211348D7
:1041F0004FF0007204F1080320604FF4800060600B
:10420000002083E80700521062619200A261CA0791
:10421000606362650A07C4E907206062C4E90A01B5
:104220002046FEF727FF2068016841F00101016088
:10423000BDE81040FF2000F005B800000038004045
:10424000F401002401B582B04FF47A70012300908C
:1042500001AA034802A9FFF72FF89DF804000EBD3C
:10426000F40100240A4A11680B6823F001030B6073
:1042700011688B6823F0E0438B6011688B680343FF
:104280008B601068016841F0010101607047000017
:10429000F401002410B502685169936943F00803E2
:1042A00093610268936943F0100393610268136895
:1042B00023F0010313600268136940F26B34A343D7
:1042C00013610268936823F44043936090F881205F
:1042D000042A0CD08A060AD5D0F8842042F0800245
:1042E000C0F884200268936943F02003936190F83A
:1042F0008120032A1DD04A060AD5D0F8842042F036
:104300000402C0F884200268936943F0400393617B
:10431000826AB2F5800F0CD10A060AD5D0F8842043
:1043200042F00202C0F884200268936943F08003DF
:1043300093618A050AD5D0F8842042F00102C0F8C2
:1043400084200268936943F400739361C9050AD518
:10435000D0F8841041F00801C0F8841001688A691F
:1043600042F480728A610021A0F86210A0F86A10FD
:1043700010BD2DE9F0411E4617460D468046069CAD
:104380000AE0601C08D024B1FDF778FC801BA04235
:1043900002D90320BDE8F081D8F80000406935EA71
:1043A000000004D00020B842EBD00020F2E701204A
:1043B000F9E770472DE9F04F93B01F4615468A463E
:1043C00004468146580700D0012000EBD7000C2F8F
:1043D00010FB07F0C0B2129003D0102F01D0182F9D
:1043E0002FD1024669462846FCF777FD002024E0DD
:1043F0001DF808600025DFF850B0300601D51C9A82
:1044000003E01D9828B9BBF8002051462046FFF76D
:1044100051FB7006641CA4B2060EA4EB0900B8425E
:1044200004D10AF101004C461FFA80FA6D1CEDB26E
:10443000082DE2D308F10100C0B2129980468842EB
:10444000D6D313B0BDE8F08F260000242DE9FF4F2E
:1044500083B09B460E46044680468A46DDE91075C9
:10446000002081461FE0B9F1000F22D005994FF0DE
:10447000000908EB0100401BA04202DA7019444613
:1044800086B20AEB0B00401BB0420FDBDDE91201E4
:104490002B463A46CDE9000131462046FFF78AFF18
:1044A000601984B2BF1C3A78002ADCD107B0BDE89D
:1044B000F08F802A01D90120D3E7059908EB01008C
:1044C000A0EB5500A04202DA7019444686B20AEB0E
:1044D0000B00401BB042E9DB0D2A0DD0DDE91201D3
:1044E0002B46CDE9000131462046FFF76BFC04EB7B
:1044F000550084B27F1CD6E77019444686B27F1CF3
:10450000F5E7000070B5284C9CB0256825F004053F
:104510002560254C00260C34256845F4404525606F
:10452000256805F440451B952568AD04FCD501249C
:1045300000940CAD03962404019402240994CDE95F
:104540000A410796082485E80D00CDE91046684623
:10455000FEF742FB88B93F2013900320CDE91406F3
:1045600040200101CDE91640CDE9180150201A90F4
:10457000022113A8FEF782F910B101201CB070BD12
:104580000A48016841F0800101600848F430016880
:1045900041F002010160006800F002001B90FDF78D
:1045A00067FA0020EAE700000C480258004402586D
:1045B000FDF76ABB1C48016841F4700101601B49AA
:1045C000086840F001000860184A002010321060AE
:1045D0000A68174B1A400A60144A18321060121DFC
:1045E0001060121D1060114A28321060121D1060F8
:1045F000121D1060121D1060121D1060121D10603F
:10460000121D1060121D10600A6822F480220A60D8
:1046100006496031086001200649C1F80801C0065A
:10462000014980390860704788ED00E00044025875
:104630007FEDF6EA0080005190F83410C90706D0EB
:1046400001684A68836B22F400321A434A6090F88A
:104650003410890706D501684A68C36B22F480329A
:104660001A434A6090F83410490706D501684A6831
:10467000036C22F480221A434A6090F83410090730
:1046800006D501684A68436C22F400421A434A6026
:1046900090F83410C90606D501688A68836C22F444
:1046A00080521A438A6090F83410890606D5016852
:1046B0008A68C36C22F400521A438A6090F834105E
:1046C000490611D501684A68036D22F480121A4325
:1046D0004A60016DB1F5801F06D101684A68436DDB
:1046E00022F4C0021A434A6090F83410090606D535
:1046F00001684A68806D22F4002202434A607047D4
:10470000F8B500250446C567FDF7B8FA07462068E6
:1047100000686FF07E46000708D500223B464FF444
:1047200000112046009600F0FBFA60B9206800688E
:1047300040070AD500223B464FF4800120460096F0
:1047400000F0EEFA08B10320F8BD202084F87900CB
:1047500084F87A00002084F87850F8BD10B5806B9A
:104760000021A0F86A10A0F86210FEF752FF10BDF9
:1047700001680A6822F490720A6001688A6822F06F
:1047800001028A60202180F87A10704710B5B0F8D5
:104790006C2090F87A300168222B05D0088B40F00D
:1047A00008000883022010BD898C8368B3F5805F00
:1047B00001D103696BB11140426E531C4366117005
:1047C000B0F86A10491E0904090CA0F86A1007D055
:1047D00015E0436E11401980416E891C4166EFE778
:1047E00001680A6822F490720A6001688A6822F0FF
:1047F00001028A60202180F87A10FFF79BF80020E0
:1048000010BD00002DE9F04F044600688025FD4BE7
:104810000021D4F810C087B0A6680F46D4F81C80D9
:1048200046EA0C06D4F814C0A26A4CEA080C46EA20
:104830000C0632430668DFF8D0C306EA0C061643BE
:10484000066020684268E66822F4405232434260C3
:104850002268A0699A4201D0266A3043A66AB6F15E
:10486000005F04D1D4E90B6C46EA0C06304396682D
:10487000DFF898C306EA0C06064396602068C26A11
:10488000666A22F00F023243C262E14E2068E14ABA
:10489000B04210D1126802F03802182A74D005DC38
:1048A000CAB3082A7AD0102A47D179E0202A7BD0CF
:1048B000282A7CD17AE0D84EB04209D1126802F0A1
:1048C0000702062A73D2DFE802F053696B6D6F713D
:1048D000D24EB04209D1126802F00702062A66D20F
:1048E000DFE802F0465C5E606264CD4EB04209D102
:1048F000126802F00702062A59D2DFE802F0394FA7
:1049000051535557C74EB0420BD1126802F00702FF
:10491000062A4CD200E00EE0DFE802F02A404244D2
:104920004648C14EB04209D1126802F03802182A36
:1049300038D0BBDCB4E74FF0010538E0BB4EB042E5
:1049400009D1126802F00702062A30D2DFE802F02D
:104950001026282A2C2EB64EB0420BD1126802F037
:104960000702062A23D2DFE802F003191B1D1F21CC
:1049700000251CE098421AD1A64A121D126802F0C6
:104980000702062A13D202E00CE007E00CE0DFE8A1
:1049900002F0030507090B0D022508E0042506E0D7
:1049A000402504E0082502E0102500E02025DFF87E
:1049B00064B2A04E9842DFF880A2ABF1540B73D1E1
:1049C000102D31D006DC022D09D0042D0AD0082D7F
:1049D0002FD111E0202D29D0402D2AD107E0FDF75D
:1049E000E3F913E06846FDF7F5F901980EE003A836
:1049F000FDF76EFA049809E0DBF8001058468906C6
:104A000010D50068C0F3C1012AFA01F0002811D0C6
:104A10006168894601EB410181420AD8B0EB093F48
:104A200007D808E05046F3E78448F1E74FF4004028
:104A3000EEE7012733E1102D4FF000084ED006DCE1
:104A4000022D0FD0042D15D0082D04D12DE0202DDE
:104A50004AD0402D13D00127794AA0F540719142E8
:104A600070D9E6E7FDF7A0F9626A0023414636F8FF
:104A700012200DE06846FDF7ADF9019803E003A8A8
:104A8000FDF726FA04980023616A36F811201946CA
:104A9000FBF71EFC62680902030241EA106150083C
:104AA000181841EB080115E032E0DBF80010584619
:104AB000890609D500680023C0F3C1012AFA01F074
:104AC000616A36F8112015E0606A002336F810207C
:104AD00050460FE00023FBF7FBFBBDE7606A0023B5
:104AE00036F81020554805E0606A002336F810209B
:104AF0004FF400400021FBF7EBFB0902020241EA00
:104B000010614FEA590010184A4641EB0801E1E7ED
:104B1000E3694FF4004293424DD1082D23D005DCC8
:104B20008DB1012D12D0042D06D112E0102D35D0FB
:104B3000202D3AD0402D11D0012721F00F00C1F3D4
:104B4000420108435AE0FDF79FFF16E0FDF7B2FF70
:104B500013E06846FDF73EF901980EE003A8FDF763
:104B6000B7F9049809E0DBF800105846890608D523
:104B70000068C0F3C1012AFA01F0616A36F8111029
:104B800010E0606A36F81010BAFBF1F0410060687E
:104B900001EB5001B1FBF0F081B2CEE7606A36F86C
:104BA00010102648B0FBF1F0F0E7606A36F810000C
:104BB000B2FBF0F0EAE7082D4AD00ADC0DB3012D74
:104BC00043D0042D7FF44DAF6846FDF703F90198FB
:104BD00009E0102D52D0202D55D0402DF2D103A840
:104BE000FDF776F90498616A36F81110B0FBF1F11F
:104BF000606801EB5001B1FBF0F080B22168C86041
:104C00004DE01FE0000C0058F369FFCFFFF4FF11E7
:104C10000010014054440258004400400048004045
:104C2000004C00400050004000140140007800405B
:104C3000007C0040045900080090D00300093D00AA
:104C4000FFFC0F00FDF720FFCDE7FDF733FFCAE7BC
:104C5000DBF80020594692060AD50968C1F3C10263
:104C60002AFA02F1626A36F81220B1FBF2F20FE082
:104C7000616A36F81120BAFBF2F209E0616A36F88F
:104C800011200949F1E7616A36F81110B2FBF1F21F
:104C9000616802EB5102B2FBF1F189B2C16007B069
:104CA0003846BDE8F08F000000093D0090F879100B
:104CB000212901D002207047B0F8621021B181682B
:104CC000B1F5805F13D014E001680A68920004D542
:104CD0008A6822F400028A6003E00A6822F08002F7
:104CE0000A600068016841F0400101600CE0016960
:104CF00061B1C16D4A1CC265026809781185B0F8BE
:104D00006210491EA0F8621000207047C16D026851
:104D10000988C1F308011185C16D891CC165EEE7E1
:104D20002DE9F0411E46174688460446069D1CE0C4
:104D3000681C1AD025B1FCF7A1FF801BA84214D92A
:104D40002068016821F4D07101602068816821F039
:104D500001018160202084F8790084F87A00002025
:104D600084F878000320BDE8F0812068C16938EA42
:104D7000010004D00020B842DAD00020F3E701207F
:104D8000F9E7000070B50D4D00240D48FEF748FC12
:104D900002E0641CAC4204D80948FEF73BFC202822
:104DA000F7D1002402E0641CAC4206D80549012278
:104DB0000348FEF76BFD0028F5D170BDFFFF010031
:104DC0001001002414000024FEE700000FB4084B7B
:104DD00010B504A902AA039800F0EEF8044602A94F
:104DE000002000F080FC204610BC5DF814FB0000A1
:104DF000E75600080907090E002804DB00F1E0204F
:104E000080F80014704700F00F0000F1E02080F8F7
:104E1000141D704702E008C8121F08C1002AFAD109
:104E200070477047002001E001C1121F002AFBD12A
:104E3000704700002DE9FF5F82B00021DDE90430FA
:104E4000020DDDF840B0034318D044F61050A2F232
:104E5000FF3242431514119801281FD0A5EB0B0017
:104E6000401C5FEA000A4FF000064E4FDFF8389111
:104E7000B046504615D5CAF1000413E0119801243C
:104E80004AA3012801D16FEA0B010298119AC0E9E7
:104E90000031C0E9024206B0BDE8F09FCBF100004E
:104EA000DFE704460021404A491842EB0450CDE9AF
:104EB000001012E0E00707D032463B464046494624
:104EC000FBF713FB8046894632463B46104619469F
:104ED000FBF70BFB06460F466410002CEAD1DDE918
:104EE0000401DDE90023BAF1000F06DAFBF7FDFA51
:104EF00042464B46FBF7F9FA05E0FBF768FB4246F2
:104F00004B46FBF764FB04460E460022284BFBF79A
:104F1000E5FB03D84FF0FF30014607E00022254BA8
:104F200020463146FBF73AFAFBF7C0FB102409E0B4
:104F3000002C0ADB0A220023FBF7CAF9039B30325C
:104F40001A55641E50EA0102F2D1641C039AC4F19E
:104F500011031444119A012A03D0012208430DD1F0
:104F60000AE0084304D000204FF0110B119072E7C3
:104F7000A3EB0B056D1E0DE05B4504DD4FF0000259
:104F800005F1010504E003DA4FF00002A5F1010587
:104F9000002AECD002981199C0E90231C0E900451D
:104FA00079E70000000014400000F03F30000000EE
:104FB0000000F0430000E03F2DE9FF4F95B09B4615
:104FC0008946064600250FE2252877D1002427468A
:104FD000F84A0121059400E0044316F8013F203B04
:104FE00001FA03F01042F7D130782A2811D06FF07F
:104FF0002F033078A0F13002092A16D8059A44F020
:10500000020402EB820203EB42021044761C05907C
:10501000EFE759F8042B0592002A03DA504244F4D2
:105020000054059044F00204761C30782E2816D1E6
:1050300016F8010F44F004042A280DD06FF02F0257
:105040003078A0F13003092B09D807EB870302EB76
:105050004303C718761CF3E759F8047B761C3078B5
:105060006C280FD006DC4C2817D068280DD06A2891
:1050700014D104E0742810D07A280FD10DE044F444
:1050800000140AE044F4801401E044F440147278FF
:10509000824202D104F58014761C761C3078662892
:1050A0000BD013DC582877D009DC002875D04528B0
:1050B000F6D04628F4D047281AD19DE118E063289D
:1050C00035D0642879D0652812D195E1702873D045
:1050D00008DC6728F1D069286FD06E280DD06F28C2
:1050E00006D1B5E073282CD0752875D0782874D0F7
:1050F0005A46179990476D1C75E1C4F30250022877
:1051000009D003280DD0D9F8001004280DD00D6067
:1051100009F1040967E1D9F80010EA17C1E9005262
:10512000F6E7D9F800100D80F2E70D70F0E719F8F6
:10513000041B8DF8001000208DF80100EA460120C4
:1051400003E059F804AB4FF0FF3061074FF0000166
:1051500002D40DE008F101018846B9420FDA80451A
:10516000F8DB1AF808100029F4D108E008F1010171
:1051700088468142FADB1AF808100029F6D1059812
:105180005B46A0EB080721463846179A00F094FAD0
:10519000284400EB080507E04DE029E10DE01AF88E
:1051A000010B5A4617999047B8F10108F7D25B46B0
:1051B00021463846179A13E142E00A220092C4F3CE
:1051C00002524FF0000A022A08D059F804CB032AF1
:1051D0004FEAEC710AD00DE029E02AE009F107015D
:1051E00021F00702F2E802C1914609E00FFA8CFCB7
:1051F0004FEAEC71042A03D14FFA8CFC4FEAEC71B0
:10520000002907DA0A460021DCF1000C61EB0201FB
:105210002D2202E0220504D52B228DF80420012244
:1052200003E0E20701D02022F7E7904659E00A2187
:1052300002E010220DE010214FF0000A00910BE077
:1052400010224FF0000A44F004040827009203E003
:1052500008224FF0000A0092C4F30252022A05D03D
:1052600059F804CB0021032A08D009E009F107010D
:1052700021F00702F2E802C1914605E01FFA8CFC1A
:10528000042A01D10CF0FF0C4FF00008220728D5AA
:10529000702806D0009B83F0100353EA0A0305D060
:1052A0000EE040228DF80420012208E05CEA0102B1
:1052B00006D030228DF804208DF805000222904699
:1052C000009B83F0080353EA0A030AD15CEA010257
:1052D00001D1620705D530228DF804204FF0010876
:1052E0007F1E582804D034A003900EA802900DE031
:1052F00036A0F9E753466046009AFAF7E9FF84467C
:105300000398825C0298401E029002705CEA0100E1
:10531000F0D1029806A9081A00F1200A600702D508
:1053200024F4803400E00127574502DDA7EB0A0092
:1053300000E0002000EB0A01009005984144401A6B
:105340000590E00306D45B462146179A059800F0C5
:10535000B3F90544002706E001A85A46C05D179935
:1053600090476D1C7F1C4745F6DBE0030CD55B4680
:105370002146179A059800F09FF9054404E0302073
:105380005A46179990476D1C0099481E00900029B5
:10539000F5DC08E0029802995A460078491C02910F
:1053A000179990476D1CBAF10001AAF1010AF1DCCE
:1053B00065E10000092801003031323334353637D9
:1053C0003839616263646566000000003031323351
:1053D00034353637383941424344454600000000F1
:1053E00000F058F90544761C307800287FF4ECADC5
:1053F00019B02846BDE8F08F620700D4062709F1EE
:10540000070222F0070CFCE80223E14603F0004803
:105410005FEA080C02D00FF2702C0DE05FEA045C2A
:1054200002D50FF2682C07E05FEAC47C02D00FF2CD
:10543000602C01E0AFF2700C4FF0FF3823F0004316
:10544000CDF850C065280CD006DC452809D0462888
:105450001DD047283DD13DE0662818D067287ED171
:1054600038E00021112F01DB112000E0781CCDE98C
:10547000000106A90EA8FFF7DDFCDDE90F010E9A79
:1054800003910021009207F1010A04914DE04FF0D1
:1054900000400097CDE9011006A90EA8FFF7CAFC4D
:1054A000DDE90F0203920E9B11990022DDF80CA09A
:1054B0000093049211B9791C00EB010AB7EB0A00C2
:1054C00004D4C0F1FF3007F1010A0490AAEB0700F1
:1054D000019044E0012F00DA01270021112F01DDA6
:1054E000112000E03846CDE9000106A90EA8FFF71B
:1054F000A1FCDDE90F010E9A0391002104910092B5
:10550000BA4621070CD40399514500DA8A46BAF10C
:10551000010F05DD009AAAF10101515C302908D084
:10552000B84202DA10F1040F06DA0121CDE90110C8
:1055300015E0AAF10101E9E7002805DC049901441E
:105540000491AAEB000102E0411C514500DD8A46AE
:105550000499401A401C01904FF00040029020072F
:1055600004D40198504501DBCDF8048000208DF86B
:105570004F0002980DF14F07B0F1004F25D02B20BE
:105580000E9002984FF0020800280CDA4042029078
:105590002D200E9007E00A210298FAF7CAFE30315A
:1055A000029007F8011DB8F10001A8F10108F2DC32
:1055B00002980028EFD1791E0E980870307800F01C
:1055C000200040F0450007F8020D12A8C01B00F1B2
:1055D00007081498007800B1012000EB0A01019837
:1055E00001EBE07105984144401A401E0590E0032C
:1055F00006D45B462146179A059800F05DF80544ED
:105600001498007818B15A46179990476D1CE0031A
:1056100024D55B462146179A059800F04DF80544BD
:105620001CE00498002807DBDDE90301884203DD64
:105630000098405C179901E0179930205A4690472E
:10564000049805F10105401C04900198401E01904A
:1056500004D12E205A46179990476D1CBAF10001CB
:10566000AAF1010ADDDC05E017F8010B5A4617998B
:1056700090476D1CB8F10001A8F10108F4DC5B460D
:105680002146179A0598ABE62D0000002B0000007C
:10569000200000002DE9F041044600251E46174673
:1056A000880404D405E039462020B0476D1C641EF0
:1056B000F9D52846BDE8F0812DE9F04104460025E2
:1056C0001E469046C80301D5302700E020278804F5
:1056D00004D505E041463846B0476D1C641EF9D537
:1056E0002846BDE8F0810A68531C0B6010707047B3
:1056F00010B504460420FDF76BFF0148046010BD9F
:105700001000002470B5002405464FF47A7603E0BB
:10571000304600F005F8641CAC42F9D370BD0000BF
:1057200070B54FF0E02500216C69094AAB69126839
:105730005043AA699A42FCD002D2A3EB020302E0D2
:10574000A4EB02063344194413468142F1D370BDE1
:10575000100000242DED028BFBF7C0F8FCF79CFA3B
:10576000042302220521A020FEF7CCFE4FF4C870CE
:10577000FFF7BEFF4FF4E13000F0A0F8FEF7F8FBB2
:10578000FEF706F9FEF704FAFBF728FA4FF6FF706A
:10579000FEF72EF9FEF70EFC10214FF4784508466F
:1057A00027A32A46FBF746F91F222021102029A310
:1057B000FBF740F91F22302110202BA3FBF73AF909
:1057C0002E4C314E9FED2E8B14210A20FBF76EFBE1
:1057D00020802EA13148FFF7F9FA304B50210820E4
:1057E0002A46FBF73DF922882DA12C48FFF7EEFA57
:1057F0002A4B6E2178202A46FBF732F920882AA10D
:1058000000EE100A2548B8EE400B20EE080BB7EE6C
:10581000C00B84ED010AB7EEC00A53EC102BFFF762
:10582000D5FA1E4B8C2108202A46FBF719F90221D4
:105830003046FCF719FAFA20FFF764FFC4E70000CE
:10584000202053544D3332483720414443202020F8
:10585000200000002020C7B6C8EBCABDBFAAB7A26F
:10586000CDF82020200000006D63756465762E74ED
:10587000616F62616F2E636F6D0000000000002495
:105880006666666666660A3F000002584144435FEA
:105890004348313028504330293A00002800002482
:1058A0003078253458000000434831305F56444476
:1058B0003A2025352E336620560000000B490A4A4F
:1058C00010B5C1E9002000208860C86008618861C7
:1058D0000C2048610846FDF763FFBDE8104004490D
:1058E00001220248FDF7D2BF001001401001002440
:1058F000140000240000000001020304010203045C
:1059000006070809010002000400060008000A005A
:105910000C0010002000400080000001000000008A
:105920000000000000000000000000003F400000F8
:105930000000000000003000400030004000000087
:1059400009000BC03D000BC03D00090018C02440F9
:105950007FE0224031800000180024C01B000D8031
:105960003240018003801C4027401C8007400040DB
:1059700010006000000000000000000000000000B7
:1059800000001F80204040200000402020401F8059
:1059900000000000090006001F800600090000004A
:1059A000040004003F8004000400000000100060B8
:1059B00000000000000000000400040004000400D7
:1059C0000400000000000040000000000000000093
:1059D000002001C006003800400000001F80204069
:1059E000204020401F800000000010403FC00040C9
:1059F0000000000018C02140224024401840000050
:105A000010802040244024401B80000002000D0034
:105A100011003FC0014000003C802440244024404D
:105A2000238000001F802440244034400380000075
:105A30003000200027C03800200000001B802440D8
:105A4000244024401B8000001C0022C02240224031
:105A50001F8000000000000008400000000000005F
:105A600000000000046000000000000000000400CE
:105A70000A001100208040400900090009000900C7
:105A80000900000000004040208011000A000400CE
:105A90001800200023402400180000001F80204030
:105AA000274029401F400000004007C039000F0078
:105AB00001C0004020403FC0244024401B80000023
:105AC0001F802040204020403080000020403FC008
:105AD000204020401F80000020403FC024402E4036
:105AE00030C0000020403FC024402E0030000000A5
:105AF0000F001080204022403380020020403FC031
:105B0000040004003FC02040204020403FC020400F
:105B1000204000000060202020203FC02000200006
:105B200020403FC024400B0030C0204020403FC0F8
:105B300020400040004000C03FC03C0003C03C008B
:105B40003FC0000020403FC00C4023003FC0200069
:105B50001F802040204020401F80000020403FC088
:105B600024402400180000001F802140214020E034
:105B70001FA0000020403FC02440260019C0004064
:105B800018C02440244022403180000030002040D2
:105B90003FC020403000000020003F800040004017
:105BA0003F80200020003E0001C007003800200098
:105BB000380007C03C0007C038000000204039C052
:105BC000060039C0204000002000384007C038409F
:105BD00020000000304021C02640384020C0000096
:105BE000000000007FE04020402000000000700026
:105BF0000C000380004000000000402040207FE0B7
:105C00000000000000002000400020000000000014
:105C10000010001000100010001000100000000024
:105C20004000000000000000000002800540054028
:105C300003C0004020003FC0044004400380000037
:105C40000000038004400440064000000000038080
:105C5000044024403FC00040000003800540054050
:105C600003400000000004401FC0244024402000E6
:105C7000000002E0055005500650042020403FC0BF
:105C80000440040003C000400000044027C000405E
:105C90000000000000100010041027E000000000C9
:105CA00020403FC00140070004C004402040204085
:105CB0003FC000400040000007C0040007C00400CF
:105CC00003C00000044007C00440040003C00040BB
:105CD000000003800440044003800000041007F02B
:105CE000045004400380000000000380044004507E
:105CF00007F00010044007C0024004000400000048
:105D0000000006400540054004C0000000000400FB
:105D10001F80044000400000040007800040044051
:105D200007C000400400070004C001800600040012
:105D3000060001C0070001C006000000044006C0C4
:105D4000010006C0044000000410071004E00180B8
:105D5000060004000000044005C0064004400000A6
:105D60000000000004007BE0402000000000000074
:105D70000000FFF000000000000040207BE0040075
:105D80000000000040008000400020002000400093
:105D90000000000000000000000000000000000003
:105DA0000000000000001FCC000C000000000000FC
:105DB00000000800300060000800300060000000B3
:105DC000022003FC1E20022003FC1E2002200000F3
:105DD00000000E1811043FFF10840C780000000032
:105DE0000F0010840F3800C0077818840078000076
:105DF00000780F8410C411240E9800E40084000879
:105E000008006800700000000000000000000000B2
:105E100000000000000007E0181820044002000005
:105E2000000040022004181807E0000000000000F5
:105E30000240024001800FF0018002400240000059
:105E40000080008000800FF800800080008000004B
:105E50000001000D000E0000000000000000000026
:105E600000000080008000800080008000800080B2
:105E70000000000C000C000000000000000000000A
:105E800000000006001800600180060018002000D5
:105E9000000007F0080810041004080807F00000CC
:105EA0000000080408041FFC0004000400000000B7
:105EB00000000E0C10141024104411840E0C00006D
:105EC00000000C1810041104110412880C7000005A
:105ED000000000E00320042408241FFC002400002C
:105EE00000001F9810841104110410881070000025
:105EF000000007F0088811041104188800700000E1
:105F000000001C00100010FC13001C00100000001A
:105F100000000E3811441084108411440E38000023
:105F200000000700088C10441044088807F00000A7
:105F3000000000000000030C030C00000000000043
:105F40000000000000010106000000000000000049
:105F50000000008001400220041008081004000026
:105F60000220022002200220022002200220000043
:105F70000000100408080410022001400080000006
:105F800000000E001200100C106C10800F000000BA
:105F900003E00C1813E4142417C4082807D00000E9
:105FA0000004003C03C41C40074000E4001C000443
:105FB00010041FFC1104110411040E88007000006D
:105FC00003E00C1810041004100410081C1000004A
:105FD00010041FFC100410041004080807F000004F
:105FE00010041FFC1104110417C410040818000049
:105FF00010041FFC1104110017C01000080000005D
:1060000003E00C181004100410441C780040000039
:1060100010041FFC10840080008010841FFC1004FA
:106020000000100410041FFC100410040000000005
:1060300000030001100110011FFE100010000000FD
:1060400010041FFC110403801464181C10040000C9
:1060500010041FFC1004000400040004000C0000E5
:1060600010041FFC1F0000FC1F001FFC1004000098
:1060700010041FFC0C04030000E010181FFC1000AB
:1060800007F00808100410041004080807F00000C6
:1060900010041FFC10841080108010800F0000007E
:1060A00007F0081810241024101C080A07F200003A
:1060B00010041FFC1104110011C011300E0C00045B
:1060C00000000E1C11041084108410441C380000C1
:1060D0001800100010041FFC10041000180000002D
:1060E00010001FF810040004000410041FF8100032
:1060F00010001E0011E0001C007013801C00100036
:106100001FC0103C00E01F0000E0103C1FC000005A
:106110001004180C163401C001C01634180C1004F9
:1061200010001C00130400FC13041C0010000000ED
:106130000804101C1064108413041C0410180000C0
:106140000000000000007FFE40024002400200000C
:10615000000030000C0003800060001C0003000001
:1061600000004002400240027FFE000000000000EC
:10617000000000002000400040004000200000001F
:106180000001000100010001000100010001000107
:10619000000040004000200000000000000000005F
:1061A00000000098012401440144014400FC000463
:1061B00010001FFC0088010401040088007000002A
:1061C0000000007000880104010401040088000040
:1061D0000000007000880104010411081FFC000485
:1061E000000000F8014401440144014400C80000DB
:1061F0000000010401040FFC110411041100180037
:10620000000000D601290129012901C90106000069
:1062100010041FFC008401000100010400FC0004C4
:1062200000000104190419FC00040004000000002F
:106230000000000300010101190119FE0000000027
:1062400010041FFC0024004001B4010C01040000F4
:106250000000100410041FFC0004000400000000F3
:10626000010401FC0104010001FC0104010000FC27
:10627000010401FC008401000100010400FC000491
:10628000000000F8010401040104010400F800000A
:10629000010101FF00850104010400880070000075
:1062A00000000070008801040104010501FF0001E5
:1062B0000104010401FC00840104010001800000CC
:1062C000000000CC012401240124012401980000D5
:1062D00000000100010007F80104010400000000B3
:1062E000010001F8000400040004010801FC00049E
:1062F000010001800170000C0010016001800100AC
:1063000001F0010C003001C00030010C01F001006F
:1063100000000104018C00740170018C0104000074
:10632000010101810171000E00180160018001006E
:1063300000000184010C013401440184010C0000BF
:10634000000000000000000001003EFC400240028E
:106350000000000000000000FFFF0000000000003F
:106360000000400240023EFC01000000000000006E
:1063700000006000800080004000400020002000FD
:10638000000000000000000000000000000000000D
:1063900000000000000000000000000000000000FD
:1063A00000000000000000000000000000000000ED
:1063B0000000000F80380FFE380F8038000000000A
:1063C00000000000000000000000000000000100CC
:1063D000000600000C00003800003100000600003C
:1063E0000C00003800003000000000000000000039
:1063F00061800067F807F9800061800061800061BA
:10640000800061800067F807F9800061800000006B
:1064100000000000000001C0E003E0F006300804C6
:1064200018081FFFFE040E080787F00381E0000034
:106430000000000001F000060C00040408060C70C7
:1064400001F9C0000E00003BE000EC18070808044A
:106450000C180003E00000000001E00007F003F862
:1064600018041C0804170807E1D003C0E00023B09B
:10647000003C08002008000010000000000000019F
:1064800000003100003200001C000000000000008D
:1064900000000000000000000000000000000000FC
:1064A00000000000000000000000000000000000EC
:1064B0007F0001FFC00780F00C00181000042000CE
:1064C000020000000000002000021000040C001870
:1064D0000780F001FFC0007F000000000000000006
:1064E0000000000000000000000000004200006604
:1064F00000006600003C0000180003FFC000180008
:10650000003C000066000066000042000000000041
:10651000080000080000080000080000080001FF53
:10652000C000080000080000080000080000080083
:1065300000000000000100003100003200001C00DB
:10654000000000000000000000000000000000004B
:106550000000000000000000080000080000080023
:106560000008000008000008000008000008000003
:10657000080000080000000000000000000000000B
:106580003800003800003800000000000000000063
:1065900000000000000000000000000000000000FB
:1065A000000600001C000070000180000E00003892
:1065B0000000C0000700001C0000300000000000C8
:1065C000000000007F8001FFE003807006001804D7
:1065D000000804000806001803807001FFE0007F37
:1065E0008000000000000000000001000801000819
:1065F00001000803FFF807FFF8000008000008008A
:10660000000800000000000000000001C03802C0C7
:1066100058040098040118040218040418061C18F1
:1066200003F81801E0F8000000000000000000017D
:10663000C0E003C0F00400080408080408080618B5
:106640000803F41801E7F00001E00000000000007A
:10665000000000000300000D0000110000610000B8
:10666000810803010807FFF80FFFF8000108000187
:10667000080000000000000000E007FCD006080849
:10668000061008061008061008061838060FF0064F
:1066900007C0000000000000000000003F8001FF74
:1066A000E0038430020818041008041008041008DD
:1066B000071810030FF00007C000000000000000E2
:1066C000000003C0000700000600000600F80607EF
:1066D000F806180006E000070000060000000000B1
:1066E00000000001E1E003F7F0063410041808048C
:1066F0001808040C08040C0806161803F3F001C16E
:10670000E000000000000000F80003FC3003063841
:106710000402080402080402080404100308F0013B
:10672000FFC0007F0000000000000000000000002B
:106730000000000000000000703800703800703861
:106740000000000000000000000000000000000049
:10675000000000000000000000000000301A0030BF
:106760001C0000000000000000000000000000000D
:1067700000000000000000080000140000220000DB
:106780004100008080010040020020040010080049
:10679000080000000000000021000021000021008E
:1067A0000021000021000021000021000021000044
:1067B000210000210000000000000000000008008F
:1067C0000804001002002001004000808000410009
:1067D0000022000014000008000000000000000378
:1067E000C00004C000040000080038080F38080882
:1067F000380810000C300007E00003C00000000063
:10680000000000003F8000FFE0038070020F1006D0
:10681000708804C088048308047F8802C090030144
:106820002000FE400000080000180001F8003E08AB
:1068300001C20007020007E20000FE00001FC800BE
:1068400001F800003800000804000807FFF807FFFF
:10685000F8040808040808040808040808061808CA
:1068600003F41801E7F00001E00000000000000060
:106870003F8001FFE003807002001804000804005C
:10688000080400080400100600200780C000000073
:1068900004000807FFF807FFF804000804000804D4
:1068A000000804001802001003807001FFE0007F60
:1068B0008000000004000807FFF807FFF80408083C
:1068C000040808040808040808043E080400080630
:1068D000001801006000000004000807FFF807FF2F
:1068E000F8040808040800040800040800043E0036
:1068F000060000060000018000000000000000000B
:106900003F8001FFE00380700600180400080402C5
:10691000080402080203F00783F0000200000200EE
:1069200004000807FFF807FFF80408080008000043
:10693000080000080000080004080807FFF807FF27
:10694000F80400080000000000000400080400082B
:1069500004000807FFF807FFF80400080400080413
:106960000008000000000000000000000006000019
:106970000700000104000104000104000307FFFEFA
:1069800007FFFC04000004000004000004000807E6
:10699000FFF807FFF8040C08001800003E0004C7C9
:1069A000800503C80600F804003804001800000839
:1069B00004000807FFF807FFF804000800000800BB
:1069C000000800000800000800000800001800008F
:1069D0006000000004000807FFF807800807FC00BB
:1069E000007FC00003F80007C00078000780080798
:1069F000FFF807FFF804000804000807FFF8070085
:106A00000803C00000E000003800001E000007007E
:106A10000001C00400F007FFF804000000000000BF
:106A20007F8001FFE0038070060018040008040066
:106A30000806001803003001FFE0007F800000001E
:106A400004000807FFF807FFF80404080404000422
:106A50000400040400040400060C0003F80001F024
:106A600000000000000000007F8001FFE003807054
:106A70000600880400880400C806003C03003E01AC
:106A8000FFE6007F8400000004000807FFF807FF0E
:106A9000F8040808040800040C00040F00040BC0EC
:106AA0000610F003F03801E00800000800000001C3
:106AB000E0F803F030063010041808041808040C3D
:106AC00008040C080206180207F00781E000000025
:106AD0000180000600000400000400000400080714
:106AE000FFF807FFF8040008040000040000060097
:106AF0000001800004000007FFE007FFF004001819
:106B00000000080000080000080000080000080459
:106B1000001007FFE004000004000006000007E08A
:106B20000007FE00041FE00001F80000380001E04B
:106B3000043E0007C0000600000400000400000737
:106B4000E00007FFC0041FF80007C007F80007FFB8
:106B500080043FF80007C004F800070000040000AC
:106B600000000004000806001807C07805F1C800FE
:106B70003E00001F800463E80780F8060018040048
:106B80000800000004000006000007800007E0087D
:106B9000047C08001FF80007F800180804E0080744
:106BA00000000600000400000000000100080600CC
:106BB000380400F80403E8040F08047C0805F00812
:106BC00007C0080700180400600000000000000073
:106BD00000000000000000000000003FFFFE200059
:106BE000022000022000022000022000020000001B
:106BF00000000000000008000007000000C00000C6
:106C000038000006000001C000003000000E000047
:106C1000010000000000000000002000022000022F
:106C20002000022000022000023FFFFE00000000C2
:106C30000000000000000000000000000000000054
:106C400000080000100000300000200000300000AC
:106C5000100000080000000000000000000001001B
:106C6000000100000100000100000100000100001F
:106C7000010000010000010000010000010000010E
:106C800000000000000000000020000020000010B4
:106C900000001000000000000000000000000000E4
:106CA000000000000000000000F00019F8001B18B0
:106CB000002208002608002408002410003FF800E5
:106CC0001FF800000800001800000004000007FF83
:106CD000F80FFFF000181800100800200800200826
:106CE000003018001FF0000FC0000000000000007E
:106CF00007C0001FF0001830002008002008002006
:106D000008003C08001C10000060000000000000AB
:106D10000000000007C0001FF00038180020080025
:106D2000200800200804101007FFF80FFFF00000F3
:106D3000100000000000000000000007C0001FF06D
:106D40000012300022180022080022080032080039
:106D50001E10000E20000000000000002000002097
:106D60000800200801FFF803FFF8062008042008A7
:106D700004200807200003000000000000000000BD
:106D8000000E000E6E001FF30031B10020B1002094
:106D9000B1003191001F13002E1E00200E003000A4
:106DA00000000004000807FFF80FFFF800100800BB
:106DB0002000002000002008003FF8001FF800001D
:106DC000080000000000000000000020080020086B
:106DD000002008063FF8063FF80000080000080001
:106DE000000800000000000000000000000000009B
:106DF00003000003002001002001002003063FFEE5
:106E0000063FFC000000000000000000000000043D
:106E1000000807FFF80FFFF8000188000300002FAB
:106E2000C00038F8002038002008000008000000EA
:106E30000000000000000400080400080400080727
:106E4000FFF80FFFF800000800000800000800002D
:106E500000000000002008003FF8003FF800100884
:106E6000002000003FF8003FF8001008002000005C
:106E70003FF8003FF8000008000000002008003F35
:106E8000F8003FF800100800100000200000200863
:106E9000003FF8001FF8000008000000000000009C
:106EA00007C0000FF0001830003008002008002054
:106EB00008003008001830000FF00007C000000084
:106EC000000000002001003FFF003FFF0010110004
:106ED0002009002008002008003038001FF0000FB3
:106EE000C00000000000000007C0001FF0003818BC
:106EF000002008002008002009001011001FFF00DA
:106F00003FFF0000010000000020080020080020D2
:106F100008003FF8003FF8000808001008002008AB
:106F200000200000300000300000000000000000E1
:106F30000000000C78001E18003308002308002110
:106F4000080021880021980030F00038600000001F
:106F500000000000200000200000200000FFF003DF
:106F6000FFF8002008002008002008000030000082
:106F700000000000000000002000003FF0007FF84B
:106F8000000018000008000008002010003FF80072
:106F90007FF0000010000000000000002000003022
:106FA00000003C00003F800023F0000078000070EB
:106FB000002380003C000030000020000020000082
:106FC0003C00003FE00023F80000E0002700003E06
:106FD00000003FE00021F80001E0003E000020003A
:106FE000000000002008002008003838003E68003B
:106FF00027800003C8002CF8003838002018002033
:1070000008000000000000002000003003003C01E8
:10701000003F830023EC000070002380003C000050
:1070200020000020000000000000000000000038E8
:10703000080020380020F80023E8002F88003E08D0
:107040000038080020180000700000000000000058
:107050000000000000000000000000000800001414
:10706000001FF7FC300006200002000000000000B6
:107070000000000000000000000000000000000010
:107080000000FFFFFF000000000000000000000003
:107090000000000000000000000020000230000698
:1070A0001FF7FC00140000080000000000000000B2
:1070B0000000000000000000000000180000600058
:1070C0000040000040000020000010000008000008
:1070D0000400000400000C0000100000B5E70200EE
:1070E000020002007FF0421042107FF04210421076
:1070F0007FF042000208020801F800000000D7D328
:107100007FF000200040008001000200FFF8020034
:10711000020002000200020002000E000000000057
:10712000BCBC10201020102013FEFC2010201020CA
:1071300015FC18843088D048105010201050518809
:107140002606CAF501000120011001107FFC038012
:1071500005400540092011102108410401020100E9
:1071600001000100D2BA0080404027F811400140E0
:107170008278424816A81AD023502220422042503A
:10718000028800000000BEA73FE020203FE0202052
:107190003FE00000FDF885088508FDF885088508B2
:1071A000FDF8850800000000B2E200084F8828883A
:1071B0000AA88AA84AA80AA82AA82AA842284508EC
:1071C00084888888103800000000CAD440502048C5
:1071D00020400FF80040E04027402240224022207B
:1071E0002A2833A82E18000800000000B3CC0000A5
:1071F0001BF0E210221023F0F800200033F068802A
:107200006080A3F02080208027F800000000D0F2EA
:10721000020001003FF820002FF0202022402180B2
:107220003FF820882090408040808380000000004C
:10723000D1D5200010F87E20444028F87E8848A848
:1072400050A864A848A872A8845018886108000053
:107250000000C9AB100010003FE0404080807FF08C
:107260004210421042107FF04000400840083FF8B2
:1072700000000000CCEE20802FF8208027F0F410D2
:1072800027F0241027F0241027F03410CFF8022024
:10729000041000000000B3E404000200FFF808003E
:1072A000104020207FF00890088008800880108817
:1072B0002088C07800000000CEC404000200020054
:1072C000FFF810401040088008800500020005000B
:1072D00008803060C01800000000D7D6040002000B
:1072E000FFF8800880083FC0008001000200FFF81E
:1072F0000200020002000E0000000000CFD43FE0B8
:10730000202020203FE0202020203FE008804890DF
:10731000289028A008800880FFF800000000CABE5E
:1073200000003FE0000000000000FFF802001240F3
:10733000122022104208820802000E000000000005
:10734000CDBC7FF84008440847C8484854884308E3
:107350004CC8733840884C08430840887FF80000C8
:107360000000C6AC00802080208020803FF02000FC
:10737000200020003FC0204020402040404080406E
:1073800000000000B4A520403840484091F07D50F6
:10739000555055507D5055F054407C40545057F84E
:1073A0008C0800000000C3FE2220222027F8FA20CB
:1073B00027F0241027F03410E7F020802FF8214028
:1073C0002220EC1800000000CAE440804140F22076
:1073D00044108BE8A000F78824A827A834A8E7A8C1
:1073E00024A8248825B800000000C8EB0800040089
:1073F000040002000200050005000880088010401B
:10740000104020204010800800000000C8AB02009F
:1074100002000500088010402020DFD80200020092
:107420001FC0020002000200FFF800000000B3CC01
:1074300000001BF0E210221023F0F800200033F0CF
:1074400068806080A3F02080208027F80000000082
:10745000BCBC208020802080F7F02080208027E0A6
:107460003220E2202140208021402220EC18000020
:107470000000CAF50200024002200200FFF80700E7
:107480000A800A8012402220421082080200020074
:1074900000000000D6A702000200FFF80200020070
:1074A0007FE010201040088005000200050018C091
:1074B000E03800000000B3D62080208023F0F88060
:1074C000208027F828203020E7F8202022202120C3
:1074D0002020E0E000000000D7A8020002007FF0BA
:1074E00004000400FFF8080010003FE00020004006
:1074F0001C800300008000000000D7A20100408033
:10750000200017F0008080804080008017F01080FD
:107510002080208040804FF800000000C5FA204005
:1075200024402440F4482450276024403440E44060
:107530002440244025482648E43800000000B7A233
:1075400002002220221044007FF8040008000FE00F
:10755000142024404280810006C03838000000001A
:10756000B3C900A0009000807FF8408040907C90DC
:10757000449044A044A0444858A841188208000000
:107580000000B9A601000100F90023F0211021102C
:107590002110211021103910C210021004100860AF
:1075A00000000000D2C60000002000780CE479043E
:1075B000516810307E6019981A3C2FE448E408386E
:1075C000003000600000D1A100000120012003FC78
:1075D00062203420042003FC240021B0212022203A
:1075E000323E18000FE00000D4F10000000010FC53
:1075F0001304110C3DF8703E10D015907CF0503EF5
:1076000018101BFE023000200000CFEE000000002A
:1076100003FE00607C4012FC110411061136112497
:107620001F44794400C0009C01860000C4BF0000D4
:1076300000000FE03C18200820043E0460046004B1
:107640007E046004200C20081FF001800000B6CCEE
:107650000000080011FC103E3EF82D8C290449045E
:1076600009043E8C50FC10881EC811FC100E00004E
:10767000B0B400000040006012FE13023A427F44A2
:1076800010C41BFE3C987190113011A00078004C82
:107690000000C8B70000004000F878C41F8C3138E3
:1076A00021EC2126413A7DE2272225FA3D260124BC
:1076B00001040000B6A80000010001705FFC700426
:1076C00020042FF801001100113821C431003F00BF
:1076D00063E040380000B3A4000000000818086010
:1076E00008C00B001E00181C7FF01000118010E075
:1076F0001838098E0F000000B0B400000040006090
:1077000012FE13023A427F4410C41BFE3C98719053
:10771000113011A00078004C0000B7B50000000047
:1077200007F80600240014F8078C0404240826181F
:1077300025F0647C64C220801FC00000BBD800001C
:1077400000001FF030182008278C2C4428442844BF
:107750002CC427842004300C1FF803800000C7B617
:107760000100210821083FF800202220223EFF428C
:10777000229422103E10221022283E282244008209
:10778000CABD0048004400440040FFFE00400040E5
:107790003E4008400840082008220F12780A2006C0
:1077A0000002BFAA00007FFC082008200820082053
:1077B0000820FFFE082008200820082010201020A4
:1077C00020204020B7A201001110110822003FFC28
:1077D0000200040007F80A080908111010A0204050
:1077E00040A003181C06CDF800007FFC40044004B4
:1077F000421452944A54442444244A544A545294BD
:107800006104400440144008D6D00100010001008A
:1078100001003FF8210821082108210821083FF82C
:1078200021080100010001000100CEC40200010096
:107830000100FFFE101010100820082004400280F4
:1078400001000280044008203018C006B2E20004A3
:1078500027C41444145485544554455415541554A0
:107860002554E55421042284224424140808CAD44F
:10787000002820241024102007FE0020F02017E00C
:10788000112011101110151019CA170A0206000252
:1078900000000000000000000000000000000000E8
:1078A00000000000000000000000000000000000D8
:1078B0000000B4F3000000000000001800001000F9
:1078C00000100000100000100000100C3FFFFE0030
:1078D00010000018000018000034000034000022DE
:1078E0000000620000410000C1800080C001006013
:1078F00006003808001C300000000000D4BD000065
:10790000000000000300C00200B00200980260887E
:107910001F888C020FF0020C80022C887FDC880309
:107920000C901B0CD01B0C6013EE60131E64130C28
:10793000F413019C1B020C27040421D800407FFC97
:107940004007F8000000B4B400000000000003800D
:107950000803000C02E00C06300C04198C08088C9B
:1079600008008C18208C2FF08C48208C08208C0864
:10797000208C08208C08608C09C10C08080C0808B1
:107980000C08080C0C0C0C07FC7800001000000020
:10799000D0C200000000000002000801003C0133DA
:1079A000C03EC200086200044200048200049A0C37
:1079B0003FFFFE0102300102300112301FE23001B0
:1079C00002300D42301936301114302114302108A4
:1079D00030471030022030000000D2BA0000000012
:1079E00000000006001803000C020C04FDF0011951
:1079F000800111004233083222F812421812651039
:107A000004E490056AB0056A200A712008614038D4
:107A100060C01860C018616018623018641E087871
:107A200000000000BEA700000000000001004001AF
:107A3000FFC001004001004001FFC0010040010003
:107A40004001FFC00100400000001064081FE7F87B
:107A50001046081046081046081FC7F810460810C0
:107A600046081046081FC7F8104608000000C6C1A7
:107A70000000000000000800000FFFF80C00180CC8
:107A800000180FFFF80C40900C30C00C10800C1147
:107A9000100DFFF808308008308008308808309CCE
:107AA0001FFFE01020801020802060802040804058
:107AB0008080030080000000B2E2000000000000AF
:107AC00011000C09FE080D860805864801A64841EC
:107AD000B64833B64813B64815B64805B64805B695
:107AE0004805B64809A64809A64839A448182048B8
:107AF0001858081844081886081902380600180093
:107B00000000CAD40000000000000001A01001D84D
:107B10000800880C008804008400FFFE000080003C
:107B200000800400803C0280047DC00408C004087A
:107B300040040840044860048822050F34073814C4
:107B400006E01C04000E000006000000000000001B
:107B50000000000000000000000000000000000025
:107B60000000000000000000000000000000000015
:107B70000000000000000000000000000000000005
:107B800000000000000000000000000000000000F5
:107B90000000000000000000B87B00080000002486
:107BA00028000000144E0008E07B00082800002494
:107BB000680C0000244E00080000000000000000D7
:107BC0000090D0030090D0030000000000000000EF
:107BD0000100000010000000000000000000FFFF96
:040000050800029954
:00000001FF
